:020000040000FA
:1000000002EF00F00F013F0E926E000E936E000E95
:10001000946E030E956E0F0E966E000E386F000EE6
:10002000396F000E3A6F000E3B6F000E3C6F806A16
:10003000816A826A836A846A896A8A6A8B6A8C6A3C
:100040008D6A00018B8C8B82006A016A026A036AE6
:10005000046A056A066A076A086A096A0A6A0B6A14
:100060000C6A0D6A0E6A0F6A106A116A126A136AC4
:10007000146A156A166A176A186A196A1A6A1B6A74
:100080001C6A1D6A1E6A1F6A206A216A226A236A24
:10009000256A266A276A296A246A286A2A6A2B6AD4
:1000A0002C6A2D6A2E6A2F6A306A316A326A336A84
:1000B000346A356A366A376A386A396A3A6A3C6A33
:1000C0003B6A3D6A3E6A3F6A406A416A426A436AE5
:1000D000446A456A466A476A486A496A4A6A4B6A94
:1000E0004C6A4D6A4E6A4F6A516A526A536A546A40
:1000F000556A566A576A586A596A5A6A5B6A5C6AEC
:100100005D6A5E6A5F6A606B616B626B636B646B96
:10011000656B666B676B000EAA6E000EA96EA69EDD
:10012000A69CA68000000000A850116E000EAA6ECA
:10013000010EA96EA69EA69CA68000000000A850F5
:10014000126E000EAA6E020EA96EA69EA69CA68036
:1001500000000000A850136E000EAA6E030EA96ED8
:10016000A69EA69CA68000000000A850146E000E5B
:10017000AA6E040EA96EA69EA69CA6800000000092
:10018000A850156E000EAA6E050EA96EA69EA69C1E
:10019000A68000000000A850166E000EAA6E060E83
:1001A000A96EA69EA69CA68000000000A850176E0F
:1001B000000EAA6E070EA96EA69EA69CA680000041
:1001C0000000A850186E000EAA6E080EA96EA69E1A
:1001D000A69CA68000000000A850196E000EAA6E12
:1001E000090EA96EA69EA69CA68000000000A8503D
:1001F0001A6E000EAA6E0A0EA96EA69EA69CA68076
:1002000000000000A8504D6E000EAA6E0B0EA96EE5
:10021000A69EA69CA68000000000A8505F6E8B8062
:10022000E6EC36F0A7EC36F020EC35F0C00E8A6E26
:100230008C9C8C9E8C8A8C9A1FEC36F03F0E8A6EBA
:100240008C9C8C9E8C8A8C9A42EC36F08B8A23ECA8
:1002500035F0CCEC42F05FEC36F0B9EC37F0F0EC76
:1002600038F05D505E6E5F50606F1D504F6E4D50A8
:100270004E6E8C864DA442EF01F083A242EF01F056
:100280007FEC41F0B9EC37F09CEC39F0EAEC44F04B
:1002900034EC45F080B674EF01F0070E5B5CD8B427
:1002A00055EF01F05B2A76EF01F05B6A3EB676EF20
:1002B00001F01550380B5C6E380E5C5CD8B465EFFD
:1002C00001F0080E5C2667EF01F0000E5C6E155021
:1002D000C70B156E5C5015124DB29CEC41F05FECF3
:1002E00036F03E8676EF01F03E965B6A80B4A0EF72
:1002F00001F0070E5A5CD8B481EF01F05A2AA2EF40
:1003000001F05A6A3EB4A2EF01F01550380B5C6E52
:10031000000E5C5CD8B491EF01F0080E5C5E93EFC8
:1003200001F0380E5C6E1550C70B156E5C5015123F
:100330004DB29CEC41F05FEC36F03E84A2EF01F050
:100340003E945A6A4DB47AEC41F034EC45F080B2F8
:10035000C4EF01F0070E595CD8B4B2EF01F0592A8E
:10036000C6EF01F0596A3EB2C6EF01F0050E415CDE
:10037000D8B4BEEF01F0412ABFEF01F0416A42EC70
:1003800036F03E82C6EF01F03E92596A34EC45F0F9
:10039000000E415CD8B4E8EF01F0010E415CD8B426
:1003A000E3EF0AF0020E415CD8B41BEF11F0030E2C
:1003B000415CD8B464EF20F0040E415CD8B4E3EFA4
:1003C00029F0050E415CD8B493EF2FF042EF01F015
:1003D0001AEC35F0410E26EC35F0B80E3FEC35F056
:1003E000700E58EC35F0100E58EC35F0100E58EC3D
:1003F00035F0100E58EC35F0000E58EC35F058EC96
:1004000052F0000E58EC35F088EC51F0000E58EC2C
:1004100035F068EC51F0000E58EC35F088EC51F0F6
:10042000000E58EC35F0C8EC51F0000E58EC35F0E9
:1004300098EC52F0000E58EC35F088EC51F0000EBC
:1004400058EC35F058EC52F088EC54F068EC52F06F
:100450001DEC35F0400E26EC35F0B80E3FEC35F0D3
:1004600078EC52F0000E58EC35F048EC51F0000EEC
:1004700058EC35F078EC52F0000E58EC35F088EC82
:1004800052F0000E58EC35F068EC52F0000E58ECCB
:1004900035F0082A210E085CD8B454EF02F0100E93
:1004A00058EC35F049EF02F0086A700E58EC35F060
:1004B00034EC45F01AEC35F0400E26EC35F0BA0E6F
:1004C0003FEC35F01DA881EF02F088EC54F088EC89
:1004D00054F088EC54F088EC54F0000E58EC35F0F1
:1004E00088EC54F0000E58EC35F088EC54F0000E17
:1004F00058EC35F088EC54F0000E58EC35F0ABEFCA
:1005000002F01BA4CDEF02F0FF0E58EC35F0B8EC72
:1005100053F0FF0E58EC35F0C8EC53F0FF0E58ECDA
:1005200035F0FF0E58EC35F0FF0E58EC35F008ECC6
:1005300054F0FF0E58EC35F008EC53F0FF0E58EC79
:1005400035F0A8EC53F0FF0E58EC35F008EC54F001
:10055000FF0E58EC35F0082A1A0E085CD8B4B6EF36
:1005600002F0000E58EC35F0ABEF02F0086A1DEC1B
:1005700035F0400E26EC35F0BA0E3FEC35F0082A87
:10058000070E085CD8B4CAEF02F0000E58EC35F044
:10059000BFEF02F0086A54EF03F0FF0E58EC35F09D
:1005A00008EC54F0FF0E58EC35F008EC53F0FF0E59
:1005B00058EC35F0A8EC53F0FF0E58EC35F008EC91
:1005C00054F0FF0E58EC35F0000E58EC35F0000EEC
:1005D00058EC35F01BA21DEF03F0FF0E58EC35F080
:1005E000C8EC53F0FF0E58EC35F0F8EC53F0FF0E6A
:1005F00058EC35F068EC53F0FF0E58EC35F048EC51
:1006000053F0FF0E58EC35F0B8EC53F0FF0E58ECF9
:1006100035F0E8EC52F0FF0E58EC35F01DEC35F0FB
:10062000400E26EC35F0BA0E3FEC35F098EC53F066
:10063000FF0E58EC35F054EF03F0FF0E58EC35F098
:1006400008EC53F0FF0E58EC35F0C8EC53F0FF0EF9
:1006500058EC35F0D8EC53F0FF0E58EC35F068EC60
:1006600054F0FF0E58EC35F0082A0D0E085CD8B493
:100670003FEF03F0000E58EC35F034EF03F0086A5A
:100680001DEC35F0400E26EC35F0BA0E3FEC35F09F
:10069000082A070E085CD8B453EF03F0000E58EC9C
:1006A00035F048EF03F0086A1DEC35F0480E26ECF3
:1006B00035F0BA0E3FEC35F01DB876EF03F01BA60F
:1006C00076EF03F0FF0E58EC35F0D8EC53F0FF0E48
:1006D00058EC35F0F8EC53F0FF0E58EC35F0C8EC60
:1006E00053F0FF0E58EC35F082EF03F0082A140E99
:1006F000085CD8B481EF03F0000E58EC35F076EFCB
:1007000003F0086A1DEC35F05D0E26EC35F0BA0EEC
:100710003FEC35F01DB8A9EF03F01BB0A9EF03F0D3
:10072000FF0E58EC35F028EC53F0FF0E58EC35F086
:10073000A8EC53F0FF0E58EC35F0D8EC53F0FF0E58
:1007400058EC35F058EC53F0FF0E58EC35F0B5EF9F
:1007500003F0082A1A0E085CD8B4B4EF03F0000EB8
:1007600058EC35F0A9EF03F0086A1AEC35F0400EAA
:1007700026EC35F0B90E3FEC35F01DB834EF05F03E
:100780001CB6CEEF03F01CB8FCEF03F01CBA2AEF46
:1007900004F01CBC5AEF04F034EF05F0FF0E58ECE7
:1007A00035F018EC53F0FF0E58EC35F018EC54F01F
:1007B000FF0E58EC35F008EC54F0FF0E58EC35F015
:1007C000FF0E58EC35F0FF0E08EC53F0FF0E58EC1E
:1007D00035F018EC53F0FF0E58EC35F0082A110EE6
:1007E000085CD8B4F9EF03F0000E58EC35F0EEEFEA
:1007F00003F0086A40EF05F0FF0E58EC35F018ECF6
:1008000053F0FF0E58EC35F018EC54F0FF0E58EC96
:1008100035F008EC54F0FF0E58EC35F0FF0E58ECB4
:1008200035F0FF0E98EC53F0FF0E58EC35F018EC55
:1008300053F0FF0E58EC35F0082A110E085CD8B4BE
:1008400027EF04F0000E58EC35F01CEF04F0086AB6
:1008500040EF05F0FF0E58EC35F068EC53F0FF0E5A
:1008600058EC35F028EC53F0FF0E58EC35F008EC5E
:1008700053F0FF0E58EC35F068EC4FF0FF0E58ECDB
:1008800035F018EC4FF0FF0E58EC35F098EC4FF0C7
:10089000FF0E58EC35F038EC4FF0FF0E58EC35F009
:1008A00078EC4FF0FF0E58EC35F0000E58EC35F0B8
:1008B00040EF05F0FF0E58EC35F0D8EC53F0FF0E8A
:1008C00058EC35F008EC53F0FF0E58EC35F0A8EC7E
:1008D00053F0FF0E58EC35F0000E58EC35F02B506D
:1008E000536E539E010E535CD8B494EF04F0490E3E
:1008F000535CD8B4BCEF04F0030E535CD8B4E4EFFF
:1009000004F0430E535CD8B40CEF05F0082A1E0E19
:10091000085CD8B491EF04F0000E58EC35F086EF87
:1009200004F0086A40EF05F0000E58EC35F0FF0EB9
:1009300058EC35F008EC53F0FF0E58EC35F018EC9D
:1009400053F0FF0E58EC35F088EC54F0000E58ECE4
:1009500035F088EC54F0000E58EC35F0000E58ECF1
:1009600035F0000E58EC35F0000E58EC35F0000E66
:1009700058EC35F040EF05F0000E58EC35F0FF0E66
:1009800058EC35F0A8EC53F0FF0E58EC35F018ECAD
:1009900053F0FF0E58EC35F088EC54F0000E58EC94
:1009A00035F088EC54F0000E58EC35F0000E58ECA1
:1009B00035F0000E58EC35F0000E58EC35F0000E16
:1009C00058EC35F040EF05F0000E58EC35F0FF0E16
:1009D00058EC35F018EC53F0FF0E58EC35F0E8EC1D
:1009E00052F0FF0E58EC35F018EC54F0FF0E58ECB6
:1009F00035F088EC54F0000E58EC35F0000E58EC51
:100A000035F0000E58EC35F0000E58EC35F0000EC5
:100A100058EC35F040EF05F0000E58EC35F0FF0EC5
:100A200058EC35F018EC53F0FF0E58EC35F008ECAC
:100A300053F0FF0E58EC35F008EC53F0FF0E58EC75
:100A400035F088EC54F0000E58EC35F0000E58EC00
:100A500035F0000E58EC35F0000E58EC35F0000E75
:100A600058EC35F040EF05F0082A320E085CD8B497
:100A70003FEF05F0000E58EC35F034EF05F0086A52
:100A80001AEC35F0730E26EC35F0B90E3FEC35F06C
:100A90001DB87EEF05F01CA27EEF05F0FF0E58ECAE
:100AA00035F008EC54F0FF0E58EC35F068EC53F0DC
:100AB000FF0E58EC35F01DEC35F0400E26EC35F00D
:100AC000B90E3FEC35F098EC53F0FF0E58EC35F0D2
:100AD00028EC53F0FF0E58EC35F0B8EC53F0FF0E55
:100AE00058EC35F008EC53F0FF0E58EC35F028ECDC
:100AF00053F0FF0E58EC35F09EEF05F0082A0E0E6D
:100B0000085CD8B489EF05F0000E58EC35F07EEFA4
:100B100005F0086A1DEC35F0400E26EC35F0B90EF4
:100B20003FEC35F0082A1F0E085CD8B49DEF05F0A5
:100B3000000E58EC35F092EF05F0086A1DEC35F028
:100B4000600E26EC35F0B90E3FEC35F01DB8CEEF57
:100B500005F01CA0CEEF05F0FF0E58EC35F058EC78
:100B600053F0FF0E58EC35F068EC53F0FF0E58ECE4
:100B700035F0FF0E58EC35F0FF0E58EC35F038EC40
:100B800053F0FF0E58EC35F008EC54F0FF0E58EC23
:100B900035F0000E58EC35F0DAEF05F0082A1C0E9F
:100BA000085CD8B4D9EF05F0000E58EC35F0CEEF64
:100BB00005F0086A1AEC35F0400E26EC35F0BB0E55
:100BC0003FEC35F04DB0EAEF05F01D504F6E506A26
:100BD000FFEF05F01D504F5CD8A43F9A000E505C0B
:100BE000D8A4F5EF05F01D504F6E3FBAFFEF05F0AA
:100BF000000E4F5CD8B4FFEF05F03EEC46F0000E5F
:100C00004F5CD8A408EF06F0BCEC46F052EF06F0BB
:100C1000400E4F5CD8A411EF06F0DCEC46F052EF2A
:100C200006F0200E4F5CD8A41AEF06F0FDEC46F05B
:100C300052EF06F0100E4F5CD8A423EF06F01EEC26
:100C400047F052EF06F0080E4F5CD8A42CEF06F0E8
:100C500056EC47F052EF06F0020E4F5CD8A435EF89
:100C600006F0A4EC47F052EF06F0010E4F5CD8A45A
:100C70003EEF06F0F2EC47F052EF06F0FF0E58ECB4
:100C800035F072EC48F04F506FEC45F0FF0E58EC29
:100C900035F0FF0E58EC35F0D1EC45F088EC54F00F
:100CA00088EC54F01AEC35F0400E26EC35F0BD0E11
:100CB0003FEC35F0000E58EC35F098EC51F0000E9A
:100CC00058EC35F068EC52F0000E58EC35F0280E78
:100CD00058EC35F0280E58EC35F0280E58EC35F06D
:100CE000280E58EC35F0280E58EC35F0000E58EC74
:100CF00035F01AEC35F0530E26EC35F0BD0E3FEC16
:100D000035F0010E625DD8A4A5EF06F0000E58EC98
:100D100035F088EC54F0000E58EC35F088EC54F0C7
:100D2000000E58EC35F0000E58EC35F0000E58EC83
:100D300035F098EC4EF0000E58EC35F088EC4EF0A3
:100D4000000E58EC35F0CEEF07F0020E625DD8A42D
:100D5000C9EF06F0000E58EC35F088EC54F0000EA8
:100D600058EC35F0A8EC4EF0000E58EC35F0A8EC3D
:100D70004EF0000E58EC35F0400E58EC35F0000EF9
:100D800058EC35F078EC4EF0000E58EC35F0CEEF24
:100D900007F0030E625DD8A4EDEF06F0000E58ECEC
:100DA00035F088EC54F0000E58EC35F088EC54F037
:100DB000000E58EC35F0000E58EC35F0000E58ECF3
:100DC00035F0A8EC4EF0000E58EC35F0E8EC4EF0A3
:100DD000000E58EC35F0CEEF07F0040E625DD8A49B
:100DE00011EF07F0000E58EC35F088EC54F0FF0ED0
:100DF00058EC35F088EC4FF0FF0E58EC35F088ECED
:100E00004FF0FF0E58EC35F0BF0E58EC35F0FF0EEA
:100E100058EC35F028EC4FF0FF0E58EC35F0CEEFE3
:100E200007F0050E625DD8A435EF07F0000E58EC10
:100E300035F088EC54F0000E58EC35F088EC54F0A6
:100E4000000E58EC35F0000E58EC35F0FF0E58EC63
:100E500035F098EC4FF0FF0E58EC35F068EC4FF0A1
:100E6000FF0E58EC35F0CEEF07F0060E625DD8A409
:100E700059EF07F0FF0E58EC35F018EC4FF0FF0E6D
:100E800058EC35F078EC4FF0FF0E58EC35F068EC8C
:100E90004FF0FF0E58EC35F0BF0E58EC35F0FF0E5A
:100EA00058EC35F048EC4FF0FF0E58EC35F0CEEF33
:100EB00007F0070E625DD8A47DEF07F0000E58EC36
:100EC00035F088EC54F0000E58EC35F0000E58EC7C
:100ED00035F0FF0E58EC35F018EC4FF0FF0E58ECE3
:100EE00035F098EC4FF0FF0E58EC35F028EC4FF051
:100EF000FF0E58EC35F0CEEF07F0000E58EC35F051
:100F0000100E58EC35F0100E58EC35F0100E58EC71
:100F100035F0100E58EC35F0100E58EC35F0000E90
:100F200058EC35F0100E58EC35F0100E58EC35F04A
:100F3000100E58EC35F0100E58EC35F0100E58EC41
:100F400035F0000E58EC35F0100E58EC35F0100E60
:100F500058EC35F0100E58EC35F0100E58EC35F01A
:100F6000100E58EC35F0000E58EC35F0400E58ECF1
:100F700035F0000E58EC35F0100E58EC35F0100E30
:100F800058EC35F0100E58EC35F0100E58EC35F0EA
:100F9000100E58EC35F0000E58EC35F0000E58EC01
:100FA00035F0E8EC51F0000E58EC35F0B8EC51F0AB
:100FB000000E58EC35F0D8EC52F0000E58EC35F03D
:100FC0001AEC35F0400E26EC35F0BC0E3FEC35F057
:100FD000000E58EC35F0C8EC51F0000E58EC35F02E
:100FE00018EC52F0000E58EC35F0280E58EC35F0A5
:100FF000280E58EC35F0280E58EC35F0280E58EC39
:1010000035F0280E58EC35F0000E58EC35F01AEC9F
:1010100035F0530E26EC35F0BC0E3FEC35F0155094
:10102000380B406E000E405CD8A43FEF08F0000E75
:1010300058EC35F058EC52F0000E58EC35F0B8ECA6
:1010400052F0000E58EC35F038EC52F0000E58EC2F
:1010500035F068EC4EF0000E58EC35F088EC54F0AA
:10106000000E58EC35F088EC54F0000E58EC35F0DA
:1010700088EC54F0000E58EC35F08AEF09F0080EB9
:10108000405CD8A46CEF08F0000E58EC35F058EC3A
:1010900052F0000E58EC35F0B8EC52F0000E58EC5F
:1010A00035F038EC52F0000E58EC35F078EC4EF09C
:1010B000000E58EC35F088EC54F0000E58EC35F08A
:1010C00088EC54F0000E58EC35F088EC54F0000E2B
:1010D00058EC35F08AEF09F0100E405CD8A499EF77
:1010E00008F0000E58EC35F058EC52F0000E58ECB9
:1010F00035F0B8EC52F0000E58EC35F038EC52F008
:10110000000E58EC35F088EC4EF0000E58EC35F03F
:1011100088EC54F0000E58EC35F088EC54F0000EDA
:1011200058EC35F088EC54F0000E58EC35F08AEFAE
:1011300009F0180E405CD8A4DDEF08F0000E58EC62
:1011400035F088EC52F0000E58EC35F068EC52F0B7
:10115000000E58EC35F058EC51F0000E58EC35F01C
:1011600088EC54F083A2C9EF08F0FF0E58EC35F07C
:10117000E8EC52F0FF0E58EC35F008EC53F0FF0E9F
:1011800058EC35F018EC54F0FF0E58EC35F08AEFBF
:1011900009F0000E58EC35F068EC52F0000E58ECF7
:1011A00035F038EC52F0000E58EC35F078EC51F098
:1011B000000E58EC35F08AEF09F0200E405CD8A400
:1011C0000AEF09F0000E58EC35F058EC52F0000E22
:1011D00058EC35F0B8EC52F0000E58EC35F038EC25
:1011E00052F0000E58EC35F0A8EC4EF0000E58EC22
:1011F00035F088EC54F0000E58EC35F088EC54F0E3
:10120000000E58EC35F088EC54F0000E58EC35F038
:101210008AEF09F0280E405CD8A437EF09F0000EE1
:1012200058EC35F058EC52F0000E58EC35F0B8ECB4
:1012300052F0000E58EC35F038EC52F0000E58EC3D
:1012400035F0B8EC4EF0000E58EC35F088EC54F068
:10125000000E58EC35F088EC54F0000E58EC35F0E8
:1012600088EC54F0000E58EC35F08AEF09F0300E9F
:10127000405CD8A464EF09F0000E58EC35F058EC4F
:1012800052F0000E58EC35F0B8EC52F0000E58EC6D
:1012900035F038EC52F0000E58EC35F0C8EC4EF05A
:1012A000000E58EC35F088EC54F0000E58EC35F098
:1012B00088EC54F0000E58EC35F088EC54F0000E39
:1012C00058EC35F08AEF09F0000E58EC35F058EC88
:1012D00052F0000E58EC35F0B8EC52F0000E58EC1D
:1012E00035F038EC52F0000E58EC35F0D8EC4EF0FA
:1012F000000E58EC35F088EC54F0000E58EC35F048
:1013000088EC54F0000E58EC35F088EC54F0000EE8
:1013100058EC35F01DA851921DB8A5EF09F0020E4A
:101320001F5CD8B4B1EF09F0030E1F5CD8B4B1EF65
:1013300009F0010E1F5CD8B4B1EF09F0210E1F5C5B
:10134000D8B4B1EF09F0ABEF09F051B2ABEF09F04F
:101350005FEC36F05182206A216A226A236A266A8B
:10136000276A20508DEC45F01AEC35F0400E26EC43
:1013700035F0BE0E3FEC35F0080E58EC35F0F80EA7
:1013800058EC35F0080E58EC35F0E00E58EC35F01E
:10139000200E58EC35F0000E58EC35F0000E58ECED
:1013A00035F0059CA9EC45F021508DEC45F01AEC88
:1013B00035F05A0E26EC35F0BE0E3FEC35F0F80E47
:1013C00058EC35F0000E58EC35F0E00E58EC35F0E6
:1013D000200E58EC35F0E00E58EC35F0000E58ECCD
:1013E00035F0000E58EC35F0059CA9EC45F0225084
:1013F0008DEC45F01AEC35F0400E26EC35F0BF0EC2
:101400003FEC35F0059CA9EC45F0A8EC54F02350D6
:101410008DEC45F01AEC35F04E0E26EC35F0BF0E93
:101420003FEC35F0059CA9EC45F026508DEC45F0DD
:101430001AEC35F05C0E26EC35F0BF0E3FEC35F0C3
:10144000059CA9EC45F0A8EC54F027508DEC45F034
:101450001AEC35F06A0E26EC35F0BF0E3FEC35F095
:10146000059CA9EC45F01DEC35F0460E26EC35F058
:10147000BC0E3FEC35F0700E58EC35F0100E58EC09
:1014800035F0100E58EC35F0100E58EC35F0000E1B
:1014900058EC35F0A8EC51F0000E58EC35F038EC73
:1014A00052F0000E58EC35F028EC52F0000E58ECDB
:1014B00035F0082A220E085CD8B464EF0AF0100E4A
:1014C00058EC35F059EF0AF0086A700E58EC35F018
:1014D0001DEC35F0460E26EC35F0BD0E3FEC35F038
:1014E000000E58EC35F068EC4EF0000E58EC35F07C
:1014F000280E58EC35F0280E58EC35F0280E58EC34
:1015000035F0280E58EC35F0280E58EC35F0000E6A
:1015100058EC35F013500F0B406E30EC3AF01DECE8
:1015200035F0460E26EC35F0BE0E3FEC35F0000EE1
:1015300058EC35F078EC4EF0000E58EC35F0280EF3
:1015400058EC35F0280E58EC35F0280E58EC35F0F4
:10155000280E58EC35F0280E58EC35F0000E58ECFB
:1015600035F01450F00B406E404240424042404241
:1015700030EC3AF01DEC35F0460E26EC35F0BF0E9F
:101580003FEC35F0000E58EC35F088EC4EF0000ED4
:1015900058EC35F0280E58EC35F0280E58EC35F0A4
:1015A000280E58EC35F0280E58EC35F0280E58EC83
:1015B00035F0000E58EC35F014500F0B406E30EC47
:1015C0003AF042EF01F0506A1AEC35F0410E26EC89
:1015D00035F0B80E3FEC35F0700E58EC35F0100ECB
:1015E00058EC35F0100E58EC35F0100E58EC35F084
:1015F000000E58EC35F068EC51F0000E58EC35F068
:1016000068EC52F0000E58EC35F0E8EC4EF0000EAD
:1016100058EC35F0A8EC4EF0000E58EC35F078ECB4
:101620004EF0000E58EC35F0C8EC4EF0000E58ECC1
:1016300035F088EC54F058EC52F0000E58EC35F0D0
:1016400088EC51F0000E58EC35F0A8EC51F01DEC90
:1016500035F0400E26EC35F0B80E3FEC35F0000EBC
:1016600058EC35F0C8EC51F0000E58EC35F068EC51
:1016700052F0000E58EC35F078EC52F0000E58ECB9
:1016800035F088EC51F0000E58EC35F058EC52F083
:10169000000E58EC35F0082A200E085CD8B456EF3E
:1016A0000BF0100E58EC35F04BEF0BF0086A700E93
:1016B00058EC35F01AEC35F0410E26EC35F0B90E49
:1016C0003FEC35F0FF0E58EC35F0E8EC52F0FF0E31
:1016D00058EC35F018EC53F0FF0E58EC35F018ECE0
:1016E00053F0FF0E58EC35F0F8EC53F0FF0E58ECC9
:1016F00035F028EC53F0FF0E58EC35F008EC54F0C0
:10170000FF0E58EC35F008EC54F0FF0E58EC35F0B5
:101710001DEC35F0410E26EC35F0B90E3FEC35F0FE
:10172000FF0E58EC35F018EC53F0FF0E58EC35F086
:10173000E8EC52F0FF0E58EC35F018EC54F0FF0EC8
:1017400058EC35F0E8EC52F0FF0E58EC35F080B074
:10175000C4EF0BF0070E565CD8B4B2EF0BF0562A6C
:10176000C6EF0BF0566A3EB0C6EF0BF0060E425CB9
:10177000D8B4BEEF0BF0422ABFEF0BF0426A42EC46
:1017800036F03E80C6EF0BF03E90566A84B6E4EF2A
:101790000BF0070E555CD8B4D1EF0BF0552AE6EFED
:1017A0000BF0556A3EBCE6EF0BF0000E425CD8B47D
:1017B000DDEF0BF04206DFEF0BF0060E426E42EC5F
:1017C00036F03E8CE6EF0BF03E9C556A34EC45F06B
:1017D0001AEC35F0410E26EC35F0BA0E3FEC35F040
:1017E000000E425CD8B415EF0CF0010E425CD8B488
:1017F000DBEF0CF0020E425CD8B4A1EF0DF0030E4B
:10180000425CD8B467EF0EF0040E425CD8B42DEF02
:101810000FF0050E425CD8B4F3EF0FF0060E425CF9
:10182000D8B4B9EF10F017EF11F068EC4EF0000EDD
:1018300058EC35F068EC4EF0000E58EC35F0B8EC92
:1018400051F0000E58EC35F01DEC35F0410E26EC51
:1018500035F0BA0E3FEC35F01150E7EC45F01AECDC
:1018600035F0410E26EC35F0BB0E3FEC35F068EC60
:101870004EF0000E58EC35F078EC4EF0000E58ECBF
:1018800035F0B8EC51F0000E58EC35F01DEC35F0A9
:10189000410E26EC35F0BB0E3FEC35F01250E7EC74
:1018A00045F01AEC35F0410E26EC35F0BC0E3FEC5D
:1018B00035F068EC4EF0000E58EC35F088EC4EF048
:1018C000000E58EC35F0B8EC51F0000E58EC35F045
:1018D0001DEC35F0410E26EC35F0BC0E3FEC35F03A
:1018E0001350E7EC45F01AEC35F0410E26EC35F0DC
:1018F000BD0E3FEC35F068EC4EF0000E58EC35F0C4
:1019000098EC4EF0000E58EC35F0B8EC51F0000EAB
:1019100058EC35F01DEC35F0410E26EC35F0BD0EDF
:101920003FEC35F01450E7EC45F01AEC35F0410E81
:1019300026EC35F0BE0E3FEC35F068EC4EF0000EB4
:1019400058EC35F0A8EC4EF0000E58EC35F0B8EC41
:1019500051F0000E58EC35F01DEC35F0410E26EC40
:1019600035F0BE0E3FEC35F01550E7EC45F01AECC3
:1019700035F0410E26EC35F0BF0E3FEC35F068EC4B
:101980004EF0000E58EC35F0B8EC4EF0000E58EC6E
:1019900035F0B8EC51F0000E58EC35F01DEC35F098
:1019A000410E26EC35F0BF0E3FEC35F01650E7EC5B
:1019B00045F017EF11F068EC4EF0000E58EC35F0E2
:1019C000C8EC4EF0000E58EC35F0B8EC51F0000EBB
:1019D00058EC35F01DEC35F0410E26EC35F0BA0E22
:1019E0003FEC35F01750E7EC45F01AEC35F0410EBE
:1019F00026EC35F0BB0E3FEC35F068EC4EF0000EF7
:101A000058EC35F0D8EC4EF0000E58EC35F0B8EC50
:101A100051F0000E58EC35F01DEC35F0410E26EC7F
:101A200035F0BB0E3FEC35F01850E7EC45F01AEC02
:101A300035F0410E26EC35F0BC0E3FEC35F068EC8D
:101A40004EF0000E58EC35F0E8EC4EF0000E58EC7D
:101A500035F0B8EC51F0000E58EC35F01DEC35F0D7
:101A6000410E26EC35F0BC0E3FEC35F01950E7EC9A
:101A700045F01AEC35F0410E26EC35F0BD0E3FEC8A
:101A800035F068EC4EF0000E58EC35F0F8EC4EF006
:101A9000000E58EC35F0B8EC51F0000E58EC35F073
:101AA0001DEC35F0410E26EC35F0BD0E3FEC35F067
:101AB0001A50E7EC45F01AEC35F0410E26EC35F003
:101AC000BE0E3FEC35F068EC4EF0000E58EC35F0F1
:101AD00048EC51F0000E58EC35F0B8EC51F0000E27
:101AE00058EC35F01DEC35F0410E26EC35F0BE0E0D
:101AF0003FEC35F01B50E7EC45F01AEC35F0410EA9
:101B000026EC35F0BF0E3FEC35F068EC4EF0000EE1
:101B100058EC35F058EC51F0000E58EC35F0B8ECBC
:101B200051F0000E58EC35F01DEC35F0410E26EC6E
:101B300035F0BF0E3FEC35F01C50E7EC45F017EFE9
:101B400011F068EC4EF0000E58EC35F068EC51F0F6
:101B5000000E58EC35F0B8EC51F0000E58EC35F0B2
:101B60001DEC35F0410E26EC35F0BA0E3FEC35F0A9
:101B70001D50E7EC45F01AEC35F0410E26EC35F03F
:101B8000BB0E3FEC35F068EC4EF0000E58EC35F033
:101B900078EC51F0000E58EC35F0B8EC51F0000E36
:101BA00058EC35F01DEC35F0410E26EC35F0BB0E4F
:101BB0003FEC35F01E50E7EC45F01AEC35F0410EE5
:101BC00026EC35F0BC0E3FEC35F068EC4EF0000E24
:101BD00058EC35F088EC51F0000E58EC35F0B8ECCC
:101BE00051F0000E58EC35F01DEC35F0410E26ECAE
:101BF00035F0BC0E3FEC35F01F50E7EC45F01AEC29
:101C000035F0410E26EC35F0BD0E3FEC35F068ECBA
:101C10004EF0000E58EC35F098EC51F0000E58ECF8
:101C200035F0B8EC51F0000E58EC35F01DEC35F005
:101C3000410E26EC35F0BD0E3FEC35F02050E7ECC0
:101C400045F01AEC35F0410E26EC35F0BE0E3FECB7
:101C500035F078EC4EF0000E58EC35F068EC4EF0B4
:101C6000000E58EC35F0B8EC51F0000E58EC35F0A1
:101C70001DEC35F0410E26EC35F0BE0E3FEC35F094
:101C80002150E7EC45F01AEC35F0410E26EC35F02A
:101C9000BF0E3FEC35F078EC4EF0000E58EC35F00E
:101CA00078EC4EF0000E58EC35F0B8EC51F0000E28
:101CB00058EC35F01DEC35F0410E26EC35F0BF0E3A
:101CC0003FEC35F02250E7EC45F017EF11F078ECDF
:101CD0004EF0000E58EC35F088EC4EF0000E58EC4B
:101CE00035F0B8EC51F0000E58EC35F01DEC35F045
:101CF000410E26EC35F0BA0E3FEC35F02350E7EC00
:101D000045F01AEC35F0410E26EC35F0BB0E3FECF9
:101D100035F078EC4EF0000E58EC35F098EC4EF0C3
:101D2000000E58EC35F0B8EC51F0000E58EC35F0E0
:101D30001DEC35F0410E26EC35F0BB0E3FEC35F0D6
:101D40002450E7EC45F01AEC35F0410E26EC35F066
:101D5000BC0E3FEC35F078EC4EF0000E58EC35F050
:101D6000A8EC4EF0000E58EC35F0B8EC51F0000E37
:101D700058EC35F01DEC35F0410E26EC35F0BC0E7C
:101D80003FEC35F02550E7EC45F01AEC35F0410E0C
:101D900026EC35F0BD0E3FEC35F078EC4EF0000E41
:101DA00058EC35F0B8EC4EF0000E58EC35F0B8ECCD
:101DB00051F0000E58EC35F01DEC35F0410E26ECDC
:101DC00035F0BD0E3FEC35F02650E7EC45F01AEC4F
:101DD00035F0410E26EC35F0BE0E3FEC35F078ECD8
:101DE0004EF0000E58EC35F0C8EC4EF0000E58ECFA
:101DF00035F0B8EC51F0000E58EC35F01DEC35F034
:101E0000410E26EC35F0BE0E3FEC35F02750E7ECE6
:101E100045F01AEC35F0410E26EC35F0BF0E3FECE4
:101E200035F078EC4EF0000E58EC35F0D8EC4EF072
:101E3000000E58EC35F0B8EC51F0000E58EC35F0CF
:101E40001DEC35F0410E26EC35F0BF0E3FEC35F0C1
:101E50002850E7EC45F017EF11F078EC4EF0000E4B
:101E600058EC35F0E8EC4EF0000E58EC35F0B8ECDC
:101E700051F0000E58EC35F01DEC35F0410E26EC1B
:101E800035F0BA0E3FEC35F02950E7EC45F01AEC8E
:101E900035F0410E26EC35F0BB0E3FEC35F078EC1A
:101EA0004EF0000E58EC35F0F8EC4EF0000E58EC09
:101EB00035F0B8EC51F0000E58EC35F01DEC35F073
:101EC000410E26EC35F0BB0E3FEC35F02A50E7EC26
:101ED00045F01AEC35F0410E26EC35F0BC0E3FEC27
:101EE00035F078EC4EF0000E58EC35F048EC51F03F
:101EF000000E58EC35F0B8EC51F0000E58EC35F00F
:101F00001DEC35F0410E26EC35F0BC0E3FEC35F003
:101F10002B50E7EC45F01AEC35F0410E26EC35F08D
:101F2000BD0E3FEC35F078EC4EF0000E58EC35F07D
:101F300058EC51F0000E58EC35F0B8EC51F0000EB2
:101F400058EC35F01DEC35F0410E26EC35F0BD0EA9
:101F50003FEC35F02C50E7EC45F01AEC35F0410E33
:101F600026EC35F0BE0E3FEC35F078EC4EF0000E6E
:101F700058EC35F068EC51F0000E58EC35F0B8EC48
:101F800051F0000E58EC35F01DEC35F0410E26EC0A
:101F900035F0BE0E3FEC35F02D50E7EC45F01AEC75
:101FA00035F0410E26EC35F0BF0E3FEC35F078EC05
:101FB0004EF0000E58EC35F078EC51F0000E58EC75
:101FC00035F0B8EC51F0000E58EC35F01DEC35F062
:101FD000410E26EC35F0BF0E3FEC35F02E50E7EC0D
:101FE00045F017EF11F078EC4EF0000E58EC35F09C
:101FF00088EC51F0000E58EC35F0B8EC51F0000EC2
:1020000058EC35F01DEC35F0410E26EC35F0BA0EEB
:102010003FEC35F02F50E7EC45F01AEC35F0410E6F
:1020200026EC35F0BB0E3FEC35F078EC4EF0000EB0
:1020300058EC35F098EC51F0000E58EC35F0B8EC57
:1020400051F0000E58EC35F01DEC35F0410E26EC49
:1020500035F0BB0E3FEC35F03050E7EC45F01AECB4
:1020600035F0410E26EC35F0BC0E3FEC35F088EC37
:102070004EF0000E58EC35F068EC4EF0000E58ECC7
:1020800035F0B8EC51F0000E58EC35F01DEC35F0A1
:10209000410E26EC35F0BC0E3FEC35F03150E7EC4C
:1020A00045F01AEC35F0410E26EC35F0BD0E3FEC54
:1020B00035F088EC4EF0000E58EC35F078EC4EF030
:1020C000000E58EC35F0B8EC51F0000E58EC35F03D
:1020D0001DEC35F0410E26EC35F0BD0E3FEC35F031
:1020E0003250E7EC45F01AEC35F0410E26EC35F0B5
:1020F000BE0E3FEC35F088EC4EF0000E58EC35F09B
:1021000088EC4EF0000E58EC35F0B8EC51F0000EB3
:1021100058EC35F01DEC35F0410E26EC35F0BE0ED6
:102120003FEC35F03350E7EC45F01AEC35F0410E5A
:1021300026EC35F0BF0E3FEC35F088EC4EF0000E8B
:1021400058EC35F098EC4EF0000E58EC35F0B8EC49
:1021500051F0000E58EC35F01DEC35F0410E26EC38
:1021600035F0BF0E3FEC35F03450E7EC45F017EF9B
:1021700011F088EC4EF0000E58EC35F0A8EC4EF063
:10218000000E58EC35F0B8EC51F0000E58EC35F07C
:102190001DEC35F0410E26EC35F0BA0E3FEC35F073
:1021A0003550E7EC45F01AEC35F0410E26EC35F0F1
:1021B000BB0E3FEC35F088EC4EF0000E58EC35F0DD
:1021C000B8EC4EF0000E58EC35F0B8EC51F0000EC3
:1021D00058EC35F01DEC35F0410E26EC35F0BB0E19
:1021E0003FEC35F03650E7EC45F01AEC35F0410E97
:1021F00026EC35F0BC0E3FEC35F088EC4EF0000ECE
:1022000058EC35F0C8EC4EF0000E58EC35F0B8EC58
:1022100051F0000E58EC35F01DEC35F0410E26EC77
:1022200035F0BC0E3FEC35F03750E7EC45F049ECAB
:1022300039F042EF01F01AEC35F0410E26EC35F0A2
:10224000B80E3FEC35F0700E58EC35F0100E58EC2F
:1022500035F0100E58EC35F0100E58EC35F0000E3D
:1022600058EC35F068EC51F0000E58EC35F068ECA5
:1022700052F0000E58EC35F0E8EC4EF0000E58EC41
:1022800035F0A8EC4EF0000E58EC35F078EC4EF03E
:10229000000E58EC35F0C8EC4EF0000E58EC35F05E
:1022A00088EC54F068EC52F0000E58EC35F088ECF5
:1022B00051F0000E58EC35F078EC52F01DEC35F092
:1022C000400E26EC35F0B80E3FEC35F0000E58EC21
:1022D00035F078EC52F0000E58EC35F0C8EC51F0C7
:1022E000000E58EC35F018EC52F0000E58EC35F0BA
:1022F000A8EC51F0000E58EC35F0082A260E085CC8
:10230000D8B488EF11F0100E58EC35F07DEF11F0D5
:10231000086A700E58EC35F034EC45F0000E435C62
:10232000D8B49AEF11F0010E435CD8B4DAEF14F090
:1023300042EF01F01AEC35F0460E26EC35F0B90EFE
:102340003FEC35F068EC52F0000E58EC35F088ECBC
:1023500051F0000E58EC35F0F8EC51F0000E58EC4E
:1023600035F088EC51F0000E58EC35F068EC51F087
:10237000000E58EC35F078EC52F0000E58EC35F0C9
:1023800088EC54F048EC51F0000E58EC35F078EC45
:1023900051F0000E58EC35F078EC51F01DEC35F0B2
:1023A000400E26EC35F0B90E3FEC35F0000E58EC3F
:1023B00035F058EC52F0000E58EC35F088EC51F046
:1023C000000E58EC35F068EC52F0000E58EC35F089
:1023D00068EC52F0000E58EC35F080B008EF12F0C7
:1023E000070E565CD8B4F8EF11F0562A0AEF12F037
:1023F000566A3EB00AEF12F00A0E465CD8B404EFFB
:1024000012F0462A05EF12F0466A3E800AEF12F0FB
:102410003E90566A84B626EF12F0070E555CD8B48B
:1024200015EF12F0552A28EF12F0556A3EBC28EF3E
:1024300012F0000E465CD8B421EF12F0460623EFEE
:1024400012F00A0E466E3E8C28EF12F03E9C556A42
:102450003F941AEC35F04A0E26EC35F0BB0E3FECFB
:1024600035F0000E465CD8B44AEF12F0000E58EC7E
:1024700035F068EC4EF0000E58EC35F068EC4EF09C
:10248000000E58EC35F0B8EC51F0000E58EC35F079
:102490005CEF12F0FF0E58EC35F008EC4FF0FF0E39
:1024A00058EC35F008EC4FF0FF0E58EC35F058ECD6
:1024B00053F0FF0E58EC35F01AEC35F0670E26ECB1
:1024C00035F0BB0E3FEC35F0010E465CD8B47DEF25
:1024D00012F0000E58EC35F068EC4EF0000E58EC9F
:1024E00035F078EC4EF0000E58EC35F0B8EC51F0C9
:1024F000000E58EC35F08FEF12F0FF0E58EC35F06F
:1025000008EC4FF0FF0E58EC35F018EC4FF0FF0ED2
:1025100058EC35F058EC53F0FF0E58EC35F01DEC4C
:1025200035F0440E26EC35F0BB0E3FEC35F0020ED4
:10253000465CD8B4B0EF12F0000E58EC35F068EC01
:102540004EF0000E58EC35F088EC4EF0000E58ECD2
:1025500035F0B8EC51F0000E58EC35F0C2EF12F047
:10256000FF0E58EC35F008EC4FF0FF0E58EC35F04C
:1025700028EC4FF0FF0E58EC35F058EC53F0FF0EFE
:1025800058EC35F01DEC35F0610E26EC35F0BB0E45
:102590003FEC35F0030E465CD8B4E3EF12F0000ECA
:1025A00058EC35F068EC4EF0000E58EC35F098EC35
:1025B0004EF0000E58EC35F0B8EC51F0000E58EC2F
:1025C00035F0F5EF12F0FF0E58EC35F008EC4FF057
:1025D000FF0E58EC35F038EC4FF0FF0E58EC35F0AC
:1025E00058EC53F0FF0E58EC35F01AEC35F04A0E6B
:1025F00026EC35F0BC0E3FEC35F0040E465CD8B44A
:1026000016EF13F0000E58EC35F068EC4EF0000EAB
:1026100058EC35F0A8EC4EF0000E58EC35F0B8EC64
:1026200051F0000E58EC35F028EF13F0FF0E58EC87
:1026300035F008EC4FF0FF0E58EC35F048EC4FF059
:10264000FF0E58EC35F058EC53F0FF0E58EC35F017
:102650001AEC35F0670E26EC35F0BC0E3FEC35F089
:10266000050E465CD8B449EF13F0000E58EC35F077
:1026700068EC4EF0000E58EC35F0B8EC4EF0000E61
:1026800058EC35F0B8EC51F0000E58EC35F05BEF3B
:1026900013F0FF0E58EC35F008EC4FF0FF0E58EC3D
:1026A00035F058EC4FF0FF0E58EC35F058EC53F085
:1026B000FF0E58EC35F01DEC35F0440E26EC35F0ED
:1026C000BC0E3FEC35F0060E465CD8B47CEF13F040
:1026D000000E58EC35F068EC4EF0000E58EC35F07A
:1026E000C8EC4EF0000E58EC35F0B8EC51F0000E8E
:1026F00058EC35F08EEF13F0FF0E58EC35F008EC87
:102700004FF0FF0E58EC35F068EC4FF0FF0E58EC30
:1027100035F058EC53F0FF0E58EC35F01DEC35F069
:10272000610E26EC35F0B40E3FEC35F0070E465C3A
:10273000D8B4AFEF13F0000E58EC35F068EC4EF063
:10274000000E58EC35F0D8EC4EF0000E58EC35F099
:10275000B8EC51F0000E58EC35F0C1EF13F0FF0E5D
:1027600058EC35F008EC4FF0FF0E58EC35F078ECF3
:102770004FF0FF0E58EC35F058EC53F0FF0E58ECCC
:1027800035F01AEC35F04A0E26EC35F0BD0E3FEC74
:1027900035F0080E465CD8B4E2EF13F0000E58ECAA
:1027A00035F068EC4EF0000E58EC35F0E8EC4EF0E9
:1027B000000E58EC35F0B8EC51F0000E58EC35F046
:1027C000F4EF13F0FF0E58EC35F008EC4FF0FF0E6D
:1027D00058EC35F088EC4FF0FF0E58EC35F058EC23
:1027E00053F0FF0E58EC35F01AEC35F0670E26EC7E
:1027F00035F0BD0E3FEC35F0090E465CD8B415EF50
:1028000014F0000E58EC35F068EC4EF0000E58EC69
:1028100035F0F8EC4EF0000E58EC35F0B8EC51F015
:10282000000E58EC35F027EF14F0FF0E58EC35F0A1
:1028300008EC4FF0FF0E58EC35F098EC4FF0FF0E1F
:1028400058EC35F058EC53F0FF0E58EC35F01AEC1C
:1028500035F04A0E26EC35F0BF0E3FEC35F00A0E8F
:10286000465CD8B47AEF14F0000E58EC35F078ECF2
:1028700051F0000E58EC35F088EC51F0000E58EC99
:1028800035F098EC51F0000E58EC35F048EC51F072
:10289000000E58EC35F088EC52F0000E58EC35F094
:1028A000F8EC51F0000E58EC35F078EC52F0000ED8
:1028B00058EC35F088EC54F0F8EC51F0000E58EC80
:1028C00035F01DEC35F0400E26EC35F0BF0E3FEC38
:1028D00035F028EC52F0000E58EC35F048EC51F091
:1028E000000E58EC35F078EC51F0000E58EC35F055
:1028F000BEEF14F0FF0E58EC35F018EC53F0FF0E5D
:1029000058EC35F028EC53F0FF0E58EC35F038EC6D
:1029100053F0FF0E58EC35F0E8EC52F0FF0E58EC97
:1029200035F028EC54F0FF0E58EC35F098EC53F0ED
:10293000FF0E58EC35F018EC54F0FF0E58EC35F063
:1029400098EC54F098EC53F0FF0E58EC35F01DEC79
:1029500035F0400E26EC35F0BF0E3FEC35F0C8ECFC
:1029600053F0FF0E58EC35F0E8EC52F0FF0E58EC47
:1029700035F018EC53F0FF0E58EC35F049EC39F017
:1029800080B8D6EF14F0070E585CD8B4CBEF14F033
:10299000582AD8EF14F0586A3EB8D8EF14F0010E58
:1029A000436E42EC36F03E88D8EF14F03E98586AF9
:1029B00042EF01F01AEC35F0460E26EC35F0B90E78
:1029C0003FEC35F0000E465CD8B416EF15F0010E62
:1029D000465CD8B417EF16F0020E465CD8B470EF20
:1029E00017F0030E465CD8B484EF18F0040E465C72
:1029F000D8B468EF19F0050E465CD8B477EF1AF03A
:102A0000060E465CD8B49EEF1BF0070E465CD8B4A9
:102A100002EF1DF0080E465CD8B4BAEF1DF0090EA7
:102A2000465CD8B472EF1EF02AEF1FF0B5EC48F008
:102A30003FB21DEF15F0050E4A6E3FB480EF15F062
:102A400080B04EEF15F0070E565CD8B42BEF15F0A2
:102A5000562A50EF15F0566A3EB050EF15F0010EB1
:102A60004A5CD8A438EF15F0080E4A6E4BEF15F00B
:102A7000040E4A5CD8A441EF15F0010E4A6E4BEFEC
:102A800015F0080E4A5CD8A44AEF15F0050E4A6E00
:102A90004BEF15F04A063E8050EF15F03E90566A17
:102AA00084B67EEF15F0070E555CD8B45BEF15F0D9
:102AB000552A80EF15F0556A3EBC80EF15F0080EE0
:102AC0004A5CD8A468EF15F0010E4A6E7BEF15F052
:102AD000010E4A5CD8A471EF15F0040E4A6E7BEF2C
:102AE00015F0050E4A5CD8A47AEF15F0080E4A6E70
:102AF0007BEF15F04A2A3E8C80EF15F03E9C556A1C
:102B00001AEC35F0460E26EC35F0BC0E3FEC35F0F5
:102B1000010E4A5CD8B4BAEF15F0040E4A5CD8B482
:102B2000DDEF15F0080E4A5CD8B4FEEF15F0FF0E8D
:102B300058EC35F018EC54F0FF0E58EC35F0F8EC8A
:102B400053F0FF0E58EC35F028EC54F0FF0E58EC23
:102B500035F0B8EC53F0FF0E58EC35F008EC53F0BC
:102B6000FF0E58EC35F088EC54F0000E58EC35F0C0
:102B7000FEEF15F0FF0E58EC35F038EC53F0FF0E79
:102B800058EC35F008EC54F0FF0E58EC35F048ECFA
:102B900054F0FF0E58EC35F008EC53F0FF0E58ECF3
:102BA00035F098EC53F0FF0E58EC35F088EC53F00C
:102BB000FF0E58EC35F0FEEF15F0FF0E58EC35F037
:102BC000D8EC53F0FF0E58EC35F018EC53F0FF0E34
:102BD00058EC35F028EC54F0FF0E58EC35F0F8ECDA
:102BE00053F0FF0E58EC35F088EC54F0000E58EC22
:102BF00035F088EC54F0000E58EC35F03FB605EF98
:102C000016F03F8611504B6E4C6EC5EC3DF01DEC3E
:102C100035F0400E26EC35F0BD0E3FEC35F040505F
:102C2000FFEC45F048EC46F03F8241EF20F00EEC1F
:102C300049F03FB21EEF16F0070E4A6E3FA44BEC70
:102C40003DF01AEC35F0460E26EC35F0BC0E3FECAC
:102C500035F0000E4A5CD8B479EF16F0010E4A5CEC
:102C6000D8B4A1EF16F0020E4A5CD8B4C9EF16F042
:102C7000030E4A5CD8B4C9EF16F0040E4A5CD8B40F
:102C8000FDEF16F0050E4A5CD8B4FDEF16F0060E07
:102C90004A5CD8B431EF17F0080E4A5CD8B457EF4D
:102CA00017F0FF0E58EC35F008EC53F0FF0E58EC1F
:102CB00035F058EC53F0FF0E58EC35F008EC54F0BA
:102CC000FF0E58EC35F088EC54F0000E58EC35F05F
:102CD00088EC54F0000E58EC35F088EC54F0000EFF
:102CE00058EC35F088EC54F0000E58EC35F057EF06
:102CF00017F0FF0E58EC35F008EC54F0FF0E58ECCE
:102D000035F048EC54F0FF0E58EC35F008EC53F079
:102D1000FF0E58EC35F098EC53F0FF0E58EC35F000
:102D200088EC53F0FF0E58EC35F088EC54F0000EB0
:102D300058EC35F088EC54F0000E58EC35F057EFB5
:102D400017F0FF0E58EC35F0A8EC53F0FF0E58ECDE
:102D500035F028EC54F0FF0E58EC35F018EC54F038
:102D6000FF0E58EC35F028EC53F0FF0E58EC35F020
:102D700008EC54F0FF0E58EC35F0E8EC52F0FF0E82
:102D800058EC35F0C8EC53F0FF0E58EC35F057EF27
:102D900017F0FF0E58EC35F068EC53F0FF0E58ECCE
:102DA00035F0B8EC53F0FF0E58EC35F018EC54F059
:102DB000FF0E58EC35F0020E4A5CD8B4E7EF16F07F
:102DC00008EC4FF0FF0E58EC35F0ECEF16F018EC75
:102DD0004FF0FF0E58EC35F088EC54F0000E58EC34
:102DE00035F088EC54F0000E58EC35F088EC54F0D7
:102DF000000E58EC35F057EF17F0FF0E58EC35F099
:102E000058EC53F0FF0E58EC35F0C8EC53F0FF0EC1
:102E100058EC35F098EC53F0FF0E58EC35F018EC08
:102E200053F0FF0E58EC35F0040E4A5CD8B420EF96
:102E300017F008EC4FF0FF0E58EC35F025EF17F0C7
:102E400018EC4FF0FF0E58EC35F088EC54F0000E03
:102E500058EC35F088EC54F0000E58EC35F057EF94
:102E600017F0FF0E58EC35F0F8EC53F0FF0E58EC6D
:102E700035F0A8EC53F0FF0E58EC35F008EC53F0A9
:102E8000FF0E58EC35F088EC53F0FF0E58EC35F09F
:102E900038EC53F0FF0E58EC35F088EC54F0000E8F
:102EA00058EC35F088EC54F0000E58EC35F03FB695
:102EB0005EEF17F03F8612504B6E4C6EC5EC3DF046
:102EC0001DEC35F0400E26EC35F0BD0E3FEC35F034
:102ED0004050FFEC45F048EC46F03F8241EF20F0D7
:102EE00067EC49F03FB277EF17F0070E4A6E3FA448
:102EF0004BEC3DF01AEC35F0460E26EC35F0BC0EEE
:102F00003FEC35F0000E4A5CD8B4F1EF17F0010E3B
:102F10004A5CD8B423EF18F0020E4A5CD8B423EF11
:102F200018F0030E4A5CD8B423EF18F0080E4A5C80
:102F3000D8B46BEF18F0FF0E58EC35F048EC53F0B6
:102F4000FF0E58EC35F0D8EC53F0FF0E58EC35F08E
:102F5000C8EC53F0FF0E58EC35F008EC4FF0FF0EC4
:102F600058EC35F008EC54F0FF0E58EC35F028EC36
:102F700053F0FF0E58EC35F098EC53F0FF0E58EC80
:102F800035F0040E4A5CD8B4D7EF17F0050E4A5C52
:102F9000D8B4DEEF17F0060E4A5CD8B4E5EF17F0B0
:102FA00008EC4FF0FF0E58EC35F0EAEF17F038EC74
:102FB0004FF0FF0E58EC35F0EAEF17F028EC4FF029
:102FC000FF0E58EC35F0EAEF17F018EC4FF0FF0E5B
:102FD00058EC35F088EC54F0000E58EC35F06BEFFF
:102FE00018F0FF0E58EC35F018EC53F0FF0E58ECCB
:102FF00035F028EC53F0FF0E58EC35F018EC54F097
:10300000FF0E58EC35F008EC53F0FF0E58EC35F09D
:1030100068EC53F0FF0E58EC35F088EC54F0000EDD
:1030200058EC35F088EC54F0000E58EC35F088EC94
:1030300054F0000E58EC35F088EC54F0000E58ECCB
:1030400035F06BEF18F0FF0E58EC35F028EC53F02C
:10305000FF0E58EC35F0A8EC53F0FF0E58EC35F0AD
:10306000D8EC53F0FF0E58EC35F058EC53F0FF0E4F
:1030700058EC35F008EC53F0FF0E58EC35F0B8EC96
:1030800053F0FF0E58EC35F018EC54F0FF0E58ECEE
:1030900035F098EC53F0FF0E58EC35F0010E4A5C19
:1030A000D8B45FEF18F0020E4A5CD8B466EF18F09F
:1030B00008EC4FF0FF0E58EC35F06BEF18F028ECF1
:1030C0004FF0FF0E58EC35F06BEF18F018EC4FF0A6
:1030D000FF0E58EC35F03FB672EF18F03F861350F4
:1030E0004B6E4C6EC5EC3DF01DEC35F0400E26EC01
:1030F00035F0BD0E3FEC35F04050FFEC45F048ECAC
:1031000046F03F8241EF20F0C0EC49F03FB28BEF38
:1031100018F0070E4A6E3FA44BEC3DF01AEC35F068
:10312000460E26EC35F0BC0E3FEC35F0000E4A5C46
:10313000D8B400EF19F0010E4A5CD8B400EF19F0D2
:10314000020E4A5CD8B400EF19F0030E4A5CD8B402
:1031500000EF19F0080E4A5CD8B44FEF19F0FF0EDB
:1031600058EC35F048EC53F0FF0E58EC35F0D8EC45
:1031700053F0FF0E58EC35F0C8EC53F0FF0E58EC4E
:1031800035F028EC4FF0FF0E58EC35F008EC54F019
:10319000FF0E58EC35F028EC53F0FF0E58EC35F0EC
:1031A00098EC53F0FF0E58EC35F0040E4A5CD8B49E
:1031B000EBEF18F0050E4A5CD8B4F2EF18F0060EEB
:1031C0004A5CD8B4F9EF18F008EC4FF0FF0E58EC59
:1031D00035F04FEF19F038EC4FF0FF0E58EC35F0AA
:1031E0004FEF19F028EC4FF0FF0E58EC35F04FEF91
:1031F00019F018EC4FF0FF0E58EC35F04FEF19F0C6
:10320000FF0E58EC35F048EC53F0FF0E58EC35F05B
:10321000D8EC53F0FF0E58EC35F0C8EC53F0FF0E2D
:1032200058EC35F018EC4FF0FF0E58EC35F008EC88
:1032300054F0FF0E58EC35F028EC53F0FF0E58EC2C
:1032400035F098EC53F0FF0E58EC35F0000E4A5C68
:10325000D8B43CEF19F0010E4A5CD8B443EF19F032
:10326000020E4A5CD8B44AEF19F008EC4FF0FF0E9A
:1032700058EC35F04FEF19F038EC4FF0FF0E58ECEA
:1032800035F04FEF19F028EC4FF0FF0E58EC35F009
:103290004FEF19F018EC4FF0FF0E58EC35F03FB639
:1032A00056EF19F03F8614504B6E4C6EC5EC3DF056
:1032B0001DEC35F0400E26EC35F0BD0E3FEC35F040
:1032C0004050FFEC45F048EC46F03F8241EF20F0E3
:1032D00019EC4AF03FB26FEF19F0070E4A6E3FA4A7
:1032E0004BEC3DF01AEC35F0460E26EC35F0BC0EFA
:1032F0003FEC35F0000E4A5CD8B4A4EF19F0010E93
:103300004A5CD8B4C7EF19F0020E4A5CD8B4EAEFB1
:1033100019F0030E4A5CD8B4EAEF19F0040E4A5CC7
:10332000D8B4EAEF19F0050E4A5CD8B425EF1AF0CC
:10333000060E4A5CD8B425EF1AF0080E4A5CD8B4E1
:103340005EEF1AF025EF1AF0FF0E58EC35F0F8ECAE
:1033500053F0FF0E58EC35F028EC54F0FF0E58EC0B
:1033600035F0B8EC53F0FF0E58EC35F088EC54F023
:10337000000E58EC35F088EC54F0000E58EC35F0A7
:1033800088EC54F0000E58EC35F05EEF1AF0FF0EAA
:1033900058EC35F0F8EC53F0FF0E58EC35F058ECE3
:1033A00054F0FF0E58EC35F018EC53F0FF0E58ECCB
:1033B00035F088EC54F0000E58EC35F088EC54F001
:1033C000000E58EC35F088EC54F0000E58EC35F057
:1033D0005EEF1AF0FF0E58EC35F0F8EC53F0FF0EEC
:1033E00058EC35F058EC54F0FF0E58EC35F008EC82
:1033F00054F0FF0E58EC35F028EC53F0FF0E58EC6B
:1034000035F098EC53F0FF0E58EC35F0020E4A5CA4
:10341000D8B417EF1AF0030E4A5CD8B41EEF1AF0B6
:1034200008EC4FF0FF0E58EC35F05EEF1AF028EC88
:103430004FF0FF0E58EC35F05EEF1AF018EC4FF03D
:10344000FF0E58EC35F05EEF1AF0FF0E58EC35F039
:1034500018EC54F0FF0E58EC35F058EC54F0FF0E19
:1034600058EC35F008EC54F0FF0E58EC35F028EC31
:1034700053F0FF0E58EC35F098EC53F0FF0E58EC7B
:1034800035F0050E4A5CD8B452EF1AF0060E4A5CCD
:10349000D8B459EF1AF008EC4FF0FF0E58EC35F0A5
:1034A0005EEF1AF028EC4FF0FF0E58EC35F05EEFAF
:1034B0001AF018EC4FF0FF0E58EC35F03FB665EF00
:1034C0001AF03F8615504B6E4C6EC5EC3DF01DEC6E
:1034D00035F0400E26EC35F0BD0E3FEC35F0405097
:1034E000FFEC45F048EC46F03F8241EF20F072ECF3
:1034F0004AF03FB27EEF1AF0070E4A6E3FA44BEC43
:103500003DF01AEC35F0460E26EC35F0BC0E3FECE3
:1035100035F0080E4A5CD8B485EF1BF0FF0E58EC6E
:1035200035F008EC54F0FF0E58EC35F0C8EC53F0D1
:10353000FF0E58EC35F0000E4A5CD8B4D9EF1AF003
:10354000010E4A5CD8B4F4EF1AF0020E4A5CD8B40B
:103550000FEF1BF0030E4A5CD8B40FEF1BF0040E04
:103560004A5CD8B436EF1BF0050E4A5CD8B451EF74
:103570001BF0060E4A5CD8B46CEF1BF098EC53F0CD
:10358000FF0E58EC35F0F8EC53F0FF0E58EC35F028
:10359000D8EC53F0FF0E58EC35F0C8EC53F0FF0EAA
:1035A00058EC35F098EC53F0FF0E58EC35F085EF01
:1035B0001BF0A8EC53F0FF0E58EC35F008EC54F07B
:1035C000FF0E58EC35F088EC54F0000E58EC35F056
:1035D00088EC54F0000E58EC35F088EC54F0000EF6
:1035E00058EC35F085EF1BF008EC54F0FF0E58EC6A
:1035F00035F038EC53F0FF0E58EC35F088EC54F011
:10360000000E58EC35F088EC54F0000E58EC35F014
:1036100088EC54F0000E58EC35F085EF1BF0F8EC18
:1036200053F0FF0E58EC35F028EC53F0FF0E58EC39
:1036300035F008EC54F0FF0E58EC35F0020E4A5C01
:10364000D8B42AEF1BF008EC4FF0FF0E58EC35F021
:103650002FEF1BF018EC4FF0FF0E58EC35F088EC14
:1036600054F0000E58EC35F085EF1BF078EC53F079
:10367000FF0E58EC35F028EC54F0FF0E58EC35F006
:1036800008EC54F0FF0E58EC35F018EC54F0FF0E37
:1036900058EC35F088EC54F0000E58EC35F085EF1E
:1036A0001BF018EC53F0FF0E58EC35F028EC53F0FB
:1036B000FF0E58EC35F098EC53F0FF0E58EC35F057
:1036C00088EC54F0000E58EC35F088EC54F0000E05
:1036D00058EC35F085EF1BF008EC54F0FF0E58EC79
:1036E00035F0D8EC53F0FF0E58EC35F0C8EC53F041
:1036F000FF0E58EC35F098EC53F0FF0E58EC35F017
:1037000088EC54F0000E58EC35F03FB68CEF1BF00F
:103710003F8616504B6E4C6EC5EC3DF01DEC35F0FF
:10372000400E26EC35F0BD0E3FEC35F04050FFEC7E
:1037300045F048EC46F03F8241EF20F01BEC4BF0A7
:103740003FB2A5EF1BF0070E4A6E3FA488EC3DF098
:103750001AEC35F0460E26EC35F0BC0E3FEC35F099
:10376000010E4A5CD8B4FBEF1BF0020E4A5CD8B4E1
:1037700023EF1CF0030E4A5CD8B44BEF1CF0040E90
:103780004A5CD8B473EF1CF0050E4A5CD8B49BEFCA
:103790001CF0060E4A5CD8B4C3EF1CF0080E4A5C5D
:1037A000D8B4E9EF1CF0FF0E58EC35F0D8EC53F02C
:1037B000FF0E58EC35F0E8EC52F0FF0E58EC35F007
:1037C000F8EC53F0FF0E58EC35F0A8EC53F0FF0E78
:1037D00058EC35F088EC54F0000E58EC35F088ECDD
:1037E00054F0000E58EC35F088EC54F0000E58EC14
:1037F00035F0E9EF1CF0FF0E58EC35F0E8EC53F033
:10380000FF0E58EC35F008EC53F0FF0E58EC35F095
:10381000F8EC53F0FF0E58EC35F008EC53F0FF0EC7
:1038200058EC35F0A8EC53F0FF0E58EC35F088EC6E
:1038300054F0000E58EC35F088EC54F0000E58ECC3
:1038400035F0E9EF1CF0FF0E58EC35F008EC53F0C2
:10385000FF0E58EC35F008EC53F0FF0E58EC35F045
:10386000F8EC53F0FF0E58EC35F008EC53F0FF0E77
:1038700058EC35F0A8EC53F0FF0E58EC35F088EC1E
:1038800054F0000E58EC35F088EC54F0000E58EC73
:1038900035F0E9EF1CF0FF0E58EC35F028EC54F051
:1038A000FF0E58EC35F0B8EC53F0FF0E58EC35F045
:1038B00098EC53F0FF0E58EC35F0C8EC53F0FF0EC7
:1038C00058EC35F008EC53F0FF0E58EC35F088EC6E
:1038D00053F0FF0E58EC35F0A8EC53F0FF0E58EC07
:1038E00035F0E9EF1CF0FF0E58EC35F038EC54F0F1
:1038F000FF0E58EC35F0A8EC53F0FF0E58EC35F005
:1039000088EC54F0000E58EC35F088EC54F0000EC2
:1039100058EC35F088EC54F0000E58EC35F088EC9B
:1039200054F0000E58EC35F088EC54F0000E58ECD2
:1039300035F0E9EF1CF0FF0E58EC35F008EC53F0D1
:10394000FF0E58EC35F0C8EC53F0FF0E58EC35F094
:10395000A8EC53F0FF0E58EC35F038EC53F0FF0EA6
:1039600058EC35F0A8EC53F0FF0E58EC35F088EC2D
:1039700054F0000E58EC35F088EC54F0000E58EC82
:1039800035F0E9EF1CF0FF0E58EC35F0F8EC52F092
:10399000FF0E58EC35F068EC53F0FF0E58EC35F0A4
:1039A000D8EC53F0FF0E58EC35F0A8EC53F0FF0EB6
:1039B00058EC35F088EC54F0000E58EC35F088ECFB
:1039C00054F0000E58EC35F088EC54F0000E58EC32
:1039D00035F03FB6F0EF1CF03F8617504B6E4C6E43
:1039E000C5EC3DF01DEC35F0400E26EC35F0BD0E7B
:1039F0003FEC35F04050FFEC45F048EC46F03F829C
:103A000041EF20F0A9EC4BF03FB209EF1DF0070E9B
:103A10004A6E3FA488EC3DF01AEC35F0460E26ECD9
:103A200035F0BC0E3FEC35F0010E4A5CD8B44AEFDD
:103A30001DF0020E4A5CD8B458EF1DF0030E4A5C2C
:103A4000D8B461EF1DF0040E4A5CD8B46FEF1DF0DE
:103A5000050E4A5CD8B482EF1DF0060E4A5CD8B45D
:103A600090EF1DF0080E4A5CD8B4A1EF1DF0B5EC44
:103A70004DF0A8EC53F0FF0E58EC35F088EC54F004
:103A8000000E58EC35F088EC54F0000E58EC35F090
:103A9000A1EF1DF02AEC4DF0A8EC53F0FF0E58EC0E
:103AA00035F088EC54F0000E58EC35F0A1EF1DF025
:103AB00042EC4DF0A8EC53F0FF0E58EC35F0A1EFBE
:103AC0001DF05FEC4DF0A8EC53F0FF0E58EC35F014
:103AD00088EC54F0000E58EC35F0A1EF1DF077ECB7
:103AE0004DF0A8EC53F0FF0E58EC35F088EC54F094
:103AF000000E58EC35F088EC54F0000E58EC35F020
:103B0000A1EF1DF08AEC4DF0A8EC53F0FF0E58EC3D
:103B100035F088EC54F0000E58EC35F0A1EF1DF0B4
:103B2000A2EC4DF0A8EC53F0FF0E58EC35F088EC09
:103B300054F0000E58EC35F088EC54F0000E58ECC0
:103B400035F03FB6A8EF1DF03F8618504B6E4C6E17
:103B5000C5EC3DF01DEC35F0400E26EC35F0BD0E09
:103B60003FEC35F04050FFEC45F048EC46F03F822A
:103B700041EF20F018EC4CF03FB2C1EF1DF0070E02
:103B80004A6E3FA488EC3DF01AEC35F0460E26EC68
:103B900035F0BC0E3FEC35F0010E4A5CD8B402EFB4
:103BA0001EF0020E4A5CD8B410EF1EF0030E4A5C01
:103BB000D8B419EF1EF0040E4A5CD8B427EF1EF0FB
:103BC000050E4A5CD8B43AEF1EF0060E4A5CD8B433
:103BD00048EF1EF0080E4A5CD8B459EF1EF0B5EC61
:103BE0004DF018EC4FF0FF0E58EC35F088EC54F027
:103BF000000E58EC35F088EC54F0000E58EC35F01F
:103C000059EF1EF02AEC4DF018EC4FF0FF0E58EC77
:103C100035F088EC54F0000E58EC35F059EF1EF0FA
:103C200042EC4DF018EC4FF0FF0E58EC35F059EF28
:103C30001EF05FEC4DF018EC4FF0FF0E58EC35F035
:103C400088EC54F0000E58EC35F059EF1EF077EC8C
:103C50004DF018EC4FF0FF0E58EC35F088EC54F0B6
:103C6000000E58EC35F088EC54F0000E58EC35F0AE
:103C700059EF1EF08AEC4DF018EC4FF0FF0E58ECA7
:103C800035F088EC54F0000E58EC35F059EF1EF08A
:103C9000A2EC4DF018EC4FF0FF0E58EC35F088EC2C
:103CA00054F0000E58EC35F088EC54F0000E58EC4F
:103CB00035F03FB660EF1EF03F8619504B6E4C6EEC
:103CC000C5EC3DF01DEC35F0400E26EC35F0BD0E98
:103CD0003FEC35F04050FFEC45F048EC46F03F82B9
:103CE00041EF20F0A1EC4CF03FB279EF1EF0070E4F
:103CF0004A6E3FA488EC3DF01AEC35F0460E26ECF7
:103D000035F0BC0E3FEC35F0010E4A5CD8B4BAEF8A
:103D10001EF0020E4A5CD8B4C8EF1EF0030E4A5CD7
:103D2000D8B4D1EF1EF0040E4A5CD8B4DFEF1EF019
:103D3000050E4A5CD8B4F2EF1EF0060E4A5CD8B409
:103D400000EF1FF0080E4A5CD8B411EF1FF0B5EC7D
:103D50004DF008EC4FF0FF0E58EC35F088EC54F0C5
:103D6000000E58EC35F088EC54F0000E58EC35F0AD
:103D700011EF1FF02AEC4DF008EC4FF0FF0E58EC5D
:103D800035F088EC54F0000E58EC35F011EF1FF0D0
:103D900042EC4DF008EC4FF0FF0E58EC35F011EF0F
:103DA0001FF05FEC4DF008EC4FF0FF0E58EC35F0D3
:103DB00088EC54F0000E58EC35F011EF1FF077EC62
:103DC0004DF008EC4FF0FF0E58EC35F088EC54F055
:103DD000000E58EC35F088EC54F0000E58EC35F03D
:103DE00011EF1FF08AEC4DF008EC4FF0FF0E58EC8D
:103DF00035F088EC54F0000E58EC35F011EF1FF060
:103E0000A2EC4DF008EC4FF0FF0E58EC35F088ECCA
:103E100054F0000E58EC35F088EC54F0000E58ECDD
:103E200035F03FB618EF1FF03F861A504B6E4C6EC0
:103E3000C5EC3DF01DEC35F0400E26EC35F0BD0E26
:103E40003FEC35F04050FFEC45F048EC46F03F8247
:103E500041EF20F078EC51F0000E58EC35F088EC92
:103E600051F0000E58EC35F098EC51F0000E58EC83
:103E700035F048EC51F0000E58EC35F088EC52F07B
:103E8000000E58EC35F0F8EC51F0000E58EC35F01F
:103E900078EC52F0000E58EC35F088EC54F0F8EC69
:103EA00051F0000E58EC35F028EC52F01DEC35F0D6
:103EB000400E26EC35F0B90E3FEC35F0000E58EC14
:103EC00035F048EC51F0000E58EC35F078EC51F03C
:103ED000000E58EC35F01AEC35F0670E26EC35F094
:103EE000BC0E3FEC35F03FB08AEF1FF0000E58ECEF
:103EF00035F0C8EC52F0000E58EC35F088EC51F07B
:103F0000000E58EC35F068EC52F0000E58EC35F02D
:103F10009CEF1FF0FF0E58EC35F068EC54F0FF0EEC
:103F200058EC35F028EC53F0FF0E58EC35F008EC67
:103F300054F0FF0E58EC35F01DEC35F0440E26EC35
:103F400035F0BC0E3FEC35F03FB0BBEF1FF0FF0E7D
:103F500058EC35F0B8EC53F0FF0E58EC35F098EC17
:103F600054F0FF0E58EC35F0C8EC53F0FF0E58EC4F
:103F700035F0CDEF1FF0000E58EC35F018EC52F094
:103F8000000E58EC35F088EC54F0000E58EC35F08B
:103F900028EC52F0000E58EC35F080B0E6EF1FF040
:103FA000070E565CD8B4D8EF1FF0562AE8EF1FF082
:103FB000566A3EB0E8EF1FF03FB0E2EF1FF03F80DF
:103FC000E3EF1FF03F903E80E8EF1FF03E90566A0F
:103FD00084B601EF20F0070E555CD8B4F3EF1FF064
:103FE000552A03EF20F0556A3EBC03EF20F03FB0A6
:103FF000FDEF1FF03F80FEEF1FF03F903E8C03EF80
:1040000020F03E9C556A80B83FEF20F0070E585CC8
:10401000D8B40EEF20F0582A41EF20F0586A3EB88D
:1040200041EF20F0436A466A42EC36F03FA03BEF96
:1040300020F0080E116E040E126E4B0E136EBB0EA6
:10404000146E9B0E156E880E166E5D905D825D94EB
:104050005D965E905E825E945E967F0E176E7F0E1A
:10406000186E000E196E000E1A6E4D6A4E6A5F6A67
:10407000606B5FEC36F03F903E8842EF01F03E9877
:10408000586A3FB462EF20F080BA60EF20F0070E6C
:10409000575CD8B44FEF20F0572A62EF20F0576AF0
:1040A0003EBA42EF01F0000E436E3E8A466A42EC91
:1040B00036F03F903F923F964A6A4B6A42EF01F0DA
:1040C0003E9A576A42EF01F01AEC35F0410E26ECA9
:1040D00035F0B80E3FEC35F0700E58EC35F0100EA0
:1040E00058EC35F0100E58EC35F0100E58EC35F059
:1040F000000E58EC35F098EC51F0000E58EC35F00D
:10410000C8EC52F0000E58EC35F088EC54F0F8ECA6
:1041100051F0000E58EC35F0C8EC51F0000E58ECA0
:1041200035F018EC52F0000E58EC35F0E8EC51F098
:10413000000E58EC35F088EC54F068EC52F0000EAC
:1041400058EC35F088EC51F0000E58EC35F01DECD1
:1041500035F0400E26EC35F0B80E3FEC35F078EC3B
:1041600052F0000E58EC35F078EC52F0000E58EC9E
:1041700035F0C8EC51F0000E58EC35F018EC52F068
:10418000000E58EC35F0A8EC51F0000E58EC35F06C
:10419000082A210E085CD8B4D3EF20F0100E58EC9A
:1041A00035F0C8EF20F0086A700E58EC35F034ECAA
:1041B00045F01AEC35F0400E26EC35F0B90E3FEC28
:1041C00035F051BE47EF21F0000E495CD8A447EF0F
:1041D00021F0FF0E58EC35F038EC53F0FF0E58ECA0
:1041E00035F068EC54F0FF0E58EC35F098EC54F0D4
:1041F00098EC53F0FF0E58EC35F068EC53F0FF0EDE
:1042000058EC35F0B8EC53F0FF0E58EC35F088EC74
:1042100053F0FF0E58EC35F098EC54F048EC54F0A5
:10422000FF0E58EC35F0F8EC53F0FF0E58EC35F07B
:1042300068EC53F01DEC35F0400E26EC35F0B90E6D
:104240003FEC35F0FF0E58EC35F018EC54F0FF0E53
:1042500058EC35F028EC53F0FF0E58EC35F098ECA4
:1042600054F038EC53F0FF0E58EC35F098EC53F066
:10427000FF0E58EC35F0E8EC52F0FF0E58EC35F03C
:1042800048EC53F0FF0E58EC35F0A3EF21F0000E90
:1042900058EC35F098EC51F0000E58EC35F0C8ECC5
:1042A00052F0000E58EC35F088EC54F0F8EC51F078
:1042B000000E58EC35F0C8EC51F0000E58EC35F01B
:1042C00018EC52F0000E58EC35F0E8EC51F0000E0E
:1042D00058EC35F088EC54F0A8EC52F0000E58EC95
:1042E00035F058EC52F0000E58EC35F0C8EC51F0B7
:1042F0001DEC35F0400E26EC35F0B90E3FEC35F0F4
:10430000000E58EC35F078EC52F0000E58EC35F019
:1043100088EC51F0000E58EC35F088EC54F098EC35
:1043200051F0000E58EC35F0F8EC51F0000E58EC5E
:1043300035F048EC51F0000E58EC35F0A8EC51F097
:10434000000E58EC35F01AEC35F0430E26EC35F043
:10435000BA0E3FEC35F01E0E58EC35F0100E58EC4E
:1043600035F0100E58EC35F0100E58EC35F0100EFC
:1043700058EC35F01AEC35F0400E26EC35F0BB0E5B
:104380003FEC35F051BE3DEF22F0010E495CD8A460
:104390003DEF22F0FF0E58EC35F0E8EC52F0FF0E46
:1043A00058EC35F028EC54F0FF0E58EC35F018ECD2
:1043B00053F0FF0E58EC35F068EC53F0FF0E58EC5C
:1043C00035F0C8EC53F0FF0E58EC35F098EC54F093
:1043D00038EC53F0FF0E58EC35F0C8EC53F0FF0EFC
:1043E00058EC35F0F8EC53F0FF0E58EC35F0A8EC33
:1043F00053F0FF0E58EC35F0870E58EC35F0EB0E0D
:1044000058EC35F0ED0E58EC35F0EB0E58EC35F07D
:104410001DEC35F0400E26EC35F0BB0E3FEC35F0D0
:10442000870E58EC35F0FF0E58EC35F018EC54F0D0
:10443000FF0E58EC35F098EC54F008EC54F0FF0EF9
:1044400058EC35F028EC53F0FF0E58EC35F098ECB2
:1044500053F0FF0E58EC35F028EC53F0FF0E58ECFB
:1044600035F008EC53F0FF0E58EC35F018EC54F032
:10447000FF0E58EC35F0AEEF22F0000E58EC35F0A0
:1044800048EC51F0000E58EC35F088EC52F0000E7C
:1044900058EC35F078EC51F0000E58EC35F0C8ECE3
:1044A00051F0000E58EC35F028EC52F0000E58ECAC
:1044B00035F088EC54F098EC51F0000E58EC35F0E3
:1044C00028EC52F0000E58EC35F058EC52F0000E8B
:1044D00058EC35F008EC52F0000E58EC35F0780E40
:1044E00058EC35F0140E58EC35F0120E58EC35F04F
:1044F000140E58EC35F01DEC35F0400E26EC35F07E
:10450000BB0E3FEC35F0780E58EC35F0000E58EC51
:1045100035F078EC52F0000E58EC35F088EC54F0A1
:1045200068EC52F0000E58EC35F088EC51F0000EBB
:1045300058EC35F0F8EC51F0000E58EC35F088EC02
:1045400051F0000E58EC35F068EC51F0000E58ECCC
:1045500035F078EC52F0000E58EC35F01AEC35F0EE
:10456000430E26EC35F0BC0E3FEC35F01E0E58EC39
:1045700035F0100E58EC35F0100E58EC35F0100EEA
:1045800058EC35F0100E58EC35F01AEC35F04A0EB8
:1045900026EC35F0BA0E3FEC35F051BEFBEF22F0C1
:1045A00060A1E7EF22F0000E58EC35F028EC52F055
:1045B000000E58EC35F018EC52F0000E58EC35F0C7
:1045C00088EC54F0000E58EC35F029EF23F0000E83
:1045D00058EC35F028EC52F0000E58EC35F098EC21
:1045E00051F0000E58EC35F098EC51F0000E58ECFC
:1045F00035F029EF23F0000E495CD8A4D0EF22F06B
:1046000060A117EF23F0FF0E58EC35F0C8EC53F023
:10461000FF0E58EC35F0B8EC53F0FF0E58EC35F0C7
:1046200088EC54F0000E58EC35F029EF23F0FF0E23
:1046300058EC35F0C8EC53F0FF0E58EC35F038EC80
:1046400053F0FF0E58EC35F038EC53F0FF0E58ECF9
:1046500035F01AEC35F04A0E26EC35F0BC0E3FEC86
:1046600035F051BE0FEF25F05E500F0B616F000E5D
:10467000615DD8B46BEF23F0010E615DD8B4AEEF8D
:1046800023F0020E615DD8B4BAEF23F0030E615D32
:10469000D8B4C6EF23F0040E615DD8B409EF24F05E
:1046A000050E615DD8B415EF24F0060E615DD8B437
:1046B00021EF24F0070E615DD8B464EF24F0080EFA
:1046C000615DD8B470EF24F0090E615DD8B47CEF61
:1046D00024F0BFEF24F0000E58EC35F078EC4EF0EB
:1046E000000E58EC35F0C8EC4EF0000E58EC35F0EA
:1046F00058EC51F0000E58EC35F0000E58EC35F047
:10470000C8EC51F0000E58EC35F078EC52F088EC23
:1047100054F058EC52F0000E58EC35F0CCEC54F05C
:10472000000E58EC35F0D8EC51F0000E58EC35F096
:104730001DEC35F0400E26EC35F0BC0E3FEC35F0AC
:1047400068EC52F0000E58EC35F078EC52F0000EA8
:1047500058EC35F088EC54F0EDEF26F0000E58ECF4
:1047600035F088EC4EF0000E58EC35F068EC4EF069
:1047700075EF23F0000E58EC35F088EC4EF0000E8B
:1047800058EC35F0A8EC4EF075EF23F0000E58EC25
:1047900035F078EC4EF0000E58EC35F0C8EC4EF0E9
:1047A000000E58EC35F058EC51F0000E58EC35F096
:1047B000000E58EC35F0C8EC51F0000E58EC35F016
:1047C00078EC52F088EC54F0C8EC51F0000E58EC44
:1047D00035F0C8EC51F0000E58EC35F068EC52F0B2
:1047E000000E58EC35F01DEC35F0400E26EC35F09F
:1047F000BC0E3FEC35F088EC54F0000E58EC35F070
:1048000088EC54F0000E58EC35F088EC54F0EDEFE5
:1048100026F0000E58EC35F088EC4EF0000E58EC07
:1048200035F068EC4EF0D0EF23F0000E58EC35F088
:1048300088EC4EF0000E58EC35F0A8EC4EF0D0EFBE
:1048400023F0000E58EC35F078EC4EF0000E58ECEA
:1048500035F0C8EC4EF0000E58EC35F058EC51F045
:10486000000E58EC35F0000E58EC35F0C8EC51F065
:10487000000E58EC35F078EC52F088EC54F0F8EC7F
:1048800051F0000E58EC35F0CCEC54F0000E58EC22
:1048900035F0D8EC51F0000E58EC35F01DEC35F049
:1048A000400E26EC35F0BC0E3FEC35F068EC52F0D3
:1048B000000E58EC35F078EC52F0000E58EC35F064
:1048C00088EC54F0EDEF26F0000E58EC35F088EC53
:1048D0004EF0000E58EC35F068EC4EF02BEF24F063
:1048E000000E58EC35F088EC4EF0000E58EC35F028
:1048F000A8EC4EF02BEF24F0000E58EC35F048EC0D
:1049000051F0000E58EC35F088EC51F0000E58ECE8
:1049100035F068EC52F0000E58EC35F098EC4EF0A3
:10492000000E58EC35F088EC54F078EC51F0000EA5
:1049300058EC35F0C8EC51F0000E58EC35F058EC5E
:1049400052F0000E58EC35F088EC51F0000E58ECA7
:1049500035F01DEC35F0400E26EC35F0BC0E3FEC8A
:1049600035F068EC51F0000E58EC35F078EC52F070
:10497000000E58EC35F088EC54F0EDEF26F0000E08
:1049800058EC35F028EC52F0000E58EC35F088EC7D
:1049900052F0000E58EC35F078EC52F0000E58EC66
:1049A00035F088EC54F028EC52F0000E58EC35F05D
:1049B00098EC51F0000E58EC35F088EC54F058ECBF
:1049C00052F0000E58EC35F048EC51F0000E58EC67
:1049D00035F07E0E58EC35F01DEC35F0400E26EC2F
:1049E00035F0BC0E3FEC35F0040E58EC35F0180EE7
:1049F00058EC35F0200E58EC35F07E0E58EC35F0C2
:104A0000000E58EC35F0A8EC51F0000E58EC35F0E3
:104A100088EC51F0000E58EC35F0EDEF26F0010E69
:104A2000495CD8A434EF23F05E500F0B616F000E89
:104A3000615DD8B44BEF25F0010E615DD8B48EEF07
:104A400025F0020E615DD8B49AEF25F0030E615D8A
:104A5000D8B4A6EF25F0040E615DD8B4E9EF25F0D7
:104A6000050E615DD8B4F5EF25F0060E615DD8B492
:104A700001EF26F0070E615DD8B444EF26F0080E72
:104A8000615DD8B450EF26F0090E615DD8B45CEFDB
:104A900026F09FEF26F0FF0E58EC35F018EC4FF0A3
:104AA000FF0E58EC35F068EC4FF0FF0E58EC35F087
:104AB000F8EC52F0FF0E58EC35F0FF0E58EC35F0E4
:104AC00068EC53F0FF0E58EC35F018EC54F098EC0D
:104AD00054F0F8EC53F0FF0E58EC35F0DCEC54F0E9
:104AE000FF0E58EC35F078EC53F0FF0E58EC35F033
:104AF0001DEC35F0400E26EC35F0BC0E3FEC35F0E9
:104B000008EC54F0FF0E58EC35F018EC54F0FF0EA2
:104B100058EC35F088EC54F0EDEF26F0FF0E58EC31
:104B200035F028EC4FF0FF0E58EC35F008EC4FF064
:104B300055EF25F0FF0E58EC35F028EC4FF0FF0E46
:104B400058EC35F048EC4FF055EF25F0FF0E58ECDF
:104B500035F018EC4FF0FF0E58EC35F068EC4FF0E4
:104B6000FF0E58EC35F0F8EC52F0FF0E58EC35F033
:104B7000FF0E58EC35F068EC53F0FF0E58EC35F0B2
:104B800018EC54F098EC54F068EC53F0FF0E58EC2D
:104B900035F068EC53F0FF0E58EC35F008EC54F0AB
:104BA000FF0E58EC35F01DEC35F0400E26EC35F0DC
:104BB000BC0E3FEC35F088EC54F0000E58EC35F0AC
:104BC00088EC54F0000E58EC35F088EC54F0EDEF22
:104BD00026F0FF0E58EC35F028EC4FF0FF0E58ECA5
:104BE00035F008EC4FF0B0EF25F0FF0E58EC35F043
:104BF00028EC4FF0FF0E58EC35F048EC4FF0B0EFDA
:104C000025F0FF0E58EC35F018EC4FF0FF0E58EC85
:104C100035F068EC4FF0FF0E58EC35F0F8EC52F040
:104C2000FF0E58EC35F0FF0E58EC35F068EC53F001
:104C3000FF0E58EC35F018EC54F098EC54F098EC6A
:104C400053F0FF0E58EC35F0DCEC54F0FF0E58EC4E
:104C500035F078EC53F0FF0E58EC35F01DEC35F0E4
:104C6000400E26EC35F0BC0E3FEC35F008EC54F06D
:104C7000FF0E58EC35F018EC54F0FF0E58EC35F000
:104C800088EC54F0EDEF26F0FF0E58EC35F028ECF0
:104C90004FF0FF0E58EC35F008EC4FF00BEF26F01C
:104CA000FF0E58EC35F028EC4FF0FF0E58EC35F0C5
:104CB00048EC4FF00BEF26F0FF0E58EC35F0E8EC27
:104CC00052F0FF0E58EC35F028EC53F0FF0E58EC84
:104CD00035F008EC54F0FF0E58EC35F038EC4FF09E
:104CE000FF0E58EC35F098EC54F018EC53F0FF0E32
:104CF00058EC35F068EC53F0FF0E58EC35F0F8EC5A
:104D000053F0FF0E58EC35F028EC53F0FF0E58EC42
:104D100035F01DEC35F0400E26EC35F0BC0E3FECC6
:104D200035F008EC53F0FF0E58EC35F018EC54F069
:104D3000FF0E58EC35F088EC54F0EDEF26F0FF0E46
:104D400058EC35F0C8EC53F0FF0E58EC35F028EC79
:104D500054F0FF0E58EC35F018EC54F0FF0E58EC00
:104D600035F098EC54F0C8EC53F0FF0E58EC35F0E9
:104D700038EC53F0FF0E58EC35F098EC54F0F8ECAA
:104D800053F0FF0E58EC35F0E8EC52F0FF0E58EC03
:104D900035F0810E58EC35F01DEC35F0400E26EC68
:104DA00035F0BC0E3FEC35F0FB0E58EC35F0E70E5D
:104DB00058EC35F0DF0E58EC35F0810E58EC35F03C
:104DC000FF0E58EC35F048EC53F0FF0E58EC35F080
:104DD00028EC53F0FF0E58EC35F01AEC35F0400E8D
:104DE00026EC35F0BD0E3FEC35F051BE5EEF27F0FE
:104DF000020E495CD8A45EEF27F0FF0E58EC35F0A8
:104E0000F8EC53F0FF0E58EC35F0A8EC53F0FF0E21
:104E100058EC35F008EC53F0FF0E58EC35F088EC08
:104E200053F0FF0E58EC35F098EC54F008EC54F0C9
:104E3000FF0E58EC35F028EC53F0FF0E58EC35F02F
:104E400098EC53F0FF0E58EC35F028EC53F0FF0EC1
:104E500058EC35F008EC53F0FF0E58EC35F0FD0E31
:104E600058EC35F0FD0E58EC35F0810E58EC35F06D
:104E7000FD0E58EC35F01DEC35F0400E26EC35F00B
:104E8000BD0E3FEC35F0FD0E58EC35F098EC54F0CB
:104E9000A8EC53F0FF0E58EC35F0C8EC53F0FF0EC1
:104EA00058EC35F018EC53F0FF0E58EC35F028ECC8
:104EB00053F0FF0E58EC35F0BDEF27F0000E58EC24
:104EC00035F058EC52F0000E58EC35F008EC52F08A
:104ED000000E58EC35F068EC51F0000E58EC35F04F
:104EE000E8EC51F0000E58EC35F088EC54F068EC2A
:104EF00052F0000E58EC35F088EC51F0000E58ECF2
:104F000035F0F8EC51F0000E58EC35F088EC51F02B
:104F1000000E58EC35F068EC51F0000E58EC35F00E
:104F2000020E58EC35F0020E58EC35F07E0E58ECBF
:104F300035F0020E58EC35F01DEC35F0400E26EC45
:104F400035F0BD0E3FEC35F0020E58EC35F088EC34
:104F500054F008EC52F0000E58EC35F028EC52F00A
:104F6000000E58EC35F078EC51F0000E58EC35F0AE
:104F700088EC51F0000E58EC35F01AEC35F0430E89
:104F800026EC35F0BE0E3FEC35F01E0E58EC35F039
:104F9000100E58EC35F0100E58EC35F0100E58ECA1
:104FA00035F0100E58EC35F01AEC35F04A0E26ECC0
:104FB00035F0BE0E3FEC35F051BE28EF28F060A36F
:104FC00005EF28F0000E58EC35F048EC51F0000EDB
:104FD00058EC35F088EC52F0000E58EC35F078ECD7
:104FE00052F0000E58EC35F028EC52F0000E58EC60
:104FF00035F088EC54F0000E58EC35F088EC54F0A5
:10500000000E58EC35F074EF28F0000E58EC35F037
:1050100008EC52F0000E58EC35F048EC51F0000E60
:1050200058EC35F018EC52F0000E58EC35F088ECE6
:1050300052F0000E58EC35F048EC51F0000E58ECF0
:1050400035F0F8EC51F0000E58EC35F074EF28F024
:10505000020E495CD8A4DFEF27F060A353EF28F0DD
:10506000FF0E58EC35F0E8EC52F0FF0E58EC35F03E
:1050700028EC54F0FF0E58EC35F018EC54F0FF0E0D
:1050800058EC35F0C8EC53F0FF0E58EC35F088ECD6
:1050900054F0000E58EC35F088EC54F0000E58EC4B
:1050A00035F074EF28F0FF0E58EC35F0A8EC53F013
:1050B000FF0E58EC35F0E8EC52F0FF0E58EC35F0EE
:1050C000B8EC53F0FF0E58EC35F028EC54F0FF0E1E
:1050D00058EC35F0E8EC52F0FF0E58EC35F098EC57
:1050E00053F0FF0E58EC35F080B816EF29F0070E9C
:1050F000585CD8B47FEF28F0582A18EF29F0586A86
:105100003EB818EF29F051AE12EF29F0519E5E50D3
:105110005D6E60515F6E5E500F0B616F000E615DE2
:10512000D8B4BDEF28F0010E615DD8B4C6EF28F009
:10513000020E615DD8B4CFEF28F0030E615DD8B4E4
:10514000D8EF28F0040E615DD8B4E0EF28F0050E2A
:10515000615DD8B4E8EF28F0060E615DD8B4F0EFD9
:1051600028F0070E615DD8B4F8EF28F0080E615DF5
:10517000D8B400EF29F008EF29F016901692169493
:1051800016861698168A168E0EEF29F0169016922D
:10519000169416861688169A168E0EEF29F016901B
:1051A0001692169416861698169A168E0EEF29F0F9
:1051B00016801692168416961698168A0EEF29F007
:1051C00016801692168416961688169A0EEF29F0F7
:1051D00016801692168416961698169A0EEF29F0D7
:1051E00016901692169416961698168A0EEF29F0B7
:1051F00016901692169416961688169A0EEF29F0A7
:1052000016901692169416961698169A0EEF29F086
:1052100016901692169416961688168AFBEC36F09F
:1052200013EF29F0518E3E8818EF29F03E98586A06
:1052300051BE1FEF29F049EC39F038EF29F080BA60
:1052400036EF29F0070E575CD8B42AEF29F0572A19
:1052500038EF29F0576A3EBA38EF29F0519E5D5079
:105260005E6E5F50606F3E8A38EF29F03E9A576A53
:1052700080B08AEF29F0070E565CD8B443EF29F0CE
:10528000562A8CEF29F0566A3EB08CEF29F051BEB9
:1052900055EF29F0020E495CD8B452EF29F0492AA3
:1052A00087EF29F0496A87EF29F0000E495CD8B4EE
:1052B00061EF29F0010E495CD8B46AEF29F080EF64
:1052C00029F060A167EF29F0609187EF29F06081F4
:1052D00087EF29F05E500F0B616F0F0E615DD8B440
:1052E0007AEF29F0090E615DD8B47AEF29F05E2AD1
:1052F00087EF29F05E905E925E945E9687EF29F0CC
:1053000060A386EF29F0609387EF29F060833E80E9
:105310008CEF29F03E90566A84B6DFEF29F0070E35
:10532000555CD8B497EF29F0552AE1EF29F0556A7A
:105330003EBCE1EF29F051BEAAEF29F0000E495C16
:10534000D8B4A6EF29F04906DCEF29F0020E496E29
:10535000DCEF29F0000E495CD8B4B6EF29F0010E5D
:10536000495CD8B4BFEF29F0D5EF29F060A1BCEFBC
:1053700029F06091DCEF29F06081DCEF29F05E50CC
:105380000F0B616F0F0E615DD8B4CFEF29F0000EE7
:10539000615DD8B4CFEF29F05E06DCEF29F05E80C6
:1053A0005E925E945E86DCEF29F060A3DBEF29F06D
:1053B0006093DCEF29F060833E8CE1EF29F03E9CA6
:1053C000556A42EF01F01AEC35F0410E26EC35F04B
:1053D000B80E3FEC35F0700E58EC35F0100E58EC6E
:1053E00035F0100E58EC35F0100E58EC35F0000E7C
:1053F00058EC35F088EC51F0000E58EC35F088ECA4
:1054000051F0000E58EC35F038EC52F0000E58EC2C
:1054100035F058EC52F0000E58EC35F028EC52F014
:10542000000E58EC35F008EC52F0000E58EC35F058
:1054300088EC54F0A8EC52F0000E58EC35F058EC23
:1054400052F0000E58EC35F0C8EC51F01DEC35F080
:10545000400E26EC35F0B80E3FEC35F0000E58EC5F
:1054600035F078EC52F0000E58EC35F088EC51F045
:10547000000E58EC35F0082A320E085CD8B446EF1E
:105480002AF0100E58EC35F03BEF2AF0086A700E47
:1054900058EC35F034EC45F0000E445CD8B458EFCD
:1054A0002AF0010E445CD8B400EF2EF042EF01F078
:1054B0001AEC35F0460E26EC35F0B90E3FEC35F01F
:1054C00068EC52F0000E58EC35F088EC51F0000E0C
:1054D00058EC35F0F8EC51F0000E58EC35F088EC53
:1054E00051F0000E58EC35F068EC51F0000E58EC1D
:1054F00035F078EC52F0000E58EC35F088EC54F0B2
:1055000048EC51F0000E58EC35F078EC51F0000EFC
:1055100058EC35F078EC51F01DEC35F0400E26ECEF
:1055200035F0B90E3FEC35F0000E58EC35F058EC84
:1055300052F0000E58EC35F088EC51F0000E58ECAB
:1055400035F068EC52F0000E58EC35F068EC52F093
:10555000000E58EC35F080B0C6EF2AF0070E565C0E
:10556000D8B4B6EF2AF0562AC8EF2AF0566A3EB0F1
:10557000C8EF2AF00B0E475CD8B4C2EF2AF0472AD6
:10558000C3EF2AF0476A3E80C8EF2AF03E90566A81
:1055900084B6E4EF2AF0070E555CD8B4D3EF2AF0B6
:1055A000552AE6EF2AF0556A3EBCE6EF2AF0000ED7
:1055B000475CD8B4DFEF2AF04706E1EF2AF00B0E84
:1055C000476E3E8CE6EF2AF03E9C556A1AEC35F0A9
:1055D0004A0E26EC35F0BB0E3FEC35F0000E475C72
:1055E000D8B407EF2BF0000E58EC35F068EC4EF015
:1055F000000E58EC35F068EC4EF0000E58EC35F02B
:10560000B8EC51F0000E58EC35F019EF2BF0FF0E0E
:1056100058EC35F008EC4FF0FF0E58EC35F008EC84
:105620004FF0FF0E58EC35F058EC53F0FF0E58ECED
:1056300035F01AEC35F0670E26EC35F0BB0E3FEC7A
:1056400035F0010E475CD8B43AEF2BF0000E58EC61
:1056500035F068EC4EF0000E58EC35F078EC4EF07A
:10566000000E58EC35F0B8EC51F0000E58EC35F067
:105670004CEF2BF0FF0E58EC35F008EC4FF0FF0E1E
:1056800058EC35F018EC4FF0FF0E58EC35F058ECB4
:1056900053F0FF0E58EC35F01DEC35F0440E26ECBF
:1056A00035F0BB0E3FEC35F0020E475CD8B46DEF21
:1056B0002BF0000E58EC35F068EC4EF0000E58EC74
:1056C00035F088EC4EF0000E58EC35F0B8EC51F0A7
:1056D000000E58EC35F07FEF2BF0FF0E58EC35F054
:1056E00008EC4FF0FF0E58EC35F028EC4FF0FF0EB1
:1056F00058EC35F058EC53F0FF0E58EC35F01DEC3B
:1057000035F0610E26EC35F0BB0E3FEC35F0030EA4
:10571000475CD8B4A0EF2BF0000E58EC35F068ECE5
:105720004EF0000E58EC35F098EC4EF0000E58ECB0
:1057300035F0B8EC51F0000E58EC35F0B2EF2BF02C
:10574000FF0E58EC35F008EC4FF0FF0E58EC35F03A
:1057500038EC4FF0FF0E58EC35F058EC53F0FF0EDC
:1057600058EC35F01AEC35F04A0E26EC35F0BC0E4C
:105770003FEC35F0040E475CD8B4D3EF2BF0000EAD
:1057800058EC35F068EC4EF0000E58EC35F0A8EC13
:105790004EF0000E58EC35F0B8EC51F0000E58EC1D
:1057A00035F0E5EF2BF0FF0E58EC35F008EC4FF03C
:1057B000FF0E58EC35F048EC4FF0FF0E58EC35F08A
:1057C00058EC53F0FF0E58EC35F01AEC35F0670E3C
:1057D00026EC35F0BC0E3FEC35F0050E475CD8B436
:1057E00006EF2CF0000E58EC35F068EC4EF0000E91
:1057F00058EC35F0B8EC4EF0000E58EC35F0B8EC43
:1058000051F0000E58EC35F018EF2CF0FF0E58EC6C
:1058100035F008EC4FF0FF0E58EC35F058EC4FF037
:10582000FF0E58EC35F058EC53F0FF0E58EC35F005
:105830001DEC35F0440E26EC35F0BC0E3FEC35F097
:10584000060E475CD8B439EF2CF0000E58EC35F05A
:1058500068EC4EF0000E58EC35F0C8EC4EF0000E3F
:1058600058EC35F0B8EC51F0000E58EC35F04BEF39
:105870002CF0FF0E58EC35F008EC4FF0FF0E58EC12
:1058800035F068EC4FF0FF0E58EC35F058EC53F063
:10589000FF0E58EC35F01DEC35F0610E26EC35F0BE
:1058A000B40E3FEC35F0070E475CD8B46CEF2CF02B
:1058B000000E58EC35F068EC4EF0000E58EC35F068
:1058C000D8EC4EF0000E58EC35F0B8EC51F0000E6C
:1058D00058EC35F07EEF2CF0FF0E58EC35F008EC6C
:1058E0004FF0FF0E58EC35F078EC4FF0FF0E58EC0F
:1058F00035F058EC53F0FF0E58EC35F01AEC35F05B
:105900004A0E26EC35F0BD0E3FEC35F0080E475C34
:10591000D8B49FEF2CF0000E58EC35F068EC4EF048
:10592000000E58EC35F0E8EC4EF0000E58EC35F077
:10593000B8EC51F0000E58EC35F0B1EF2CF0FF0E42
:1059400058EC35F008EC4FF0FF0E58EC35F088ECD1
:105950004FF0FF0E58EC35F058EC53F0FF0E58ECBA
:1059600035F01AEC35F0670E26EC35F0BD0E3FEC45
:1059700035F0090E475CD8B4D2EF2CF0000E58EC8D
:1059800035F068EC4EF0000E58EC35F0F8EC4EF0C7
:10599000000E58EC35F0B8EC51F0000E58EC35F034
:1059A000E4EF2CF0FF0E58EC35F008EC4FF0FF0E52
:1059B00058EC35F098EC4FF0FF0E58EC35F058EC01
:1059C00053F0FF0E58EC35F01AEC35F04A0E26EC89
:1059D00035F0BE0E3FEC35F00A0E475CD8B420EF30
:1059E0002DF0000E58EC35F028EC52F0000E58EC7B
:1059F00035F078EC52F0000E58EC35F0B8EC51F080
:105A0000000E58EC35F088EC51F0000E58EC35F0F3
:105A100058EC52F0000E58EC35F088EC54F068EC7D
:105A200052F0000E58EC35F088EC51F0000E58ECB6
:105A300035F078EC52F0000E58EC35F04DEF2DF0CB
:105A4000FF0E58EC35F0C8EC53F0FF0E58EC35F073
:105A500018EC54F0FF0E58EC35F058EC53F0FF0EF4
:105A600058EC35F028EC53F0FF0E58EC35F0F8EC1C
:105A700053F0FF0E58EC35F098EC54F008EC54F06D
:105A8000FF0E58EC35F028EC53F0FF0E58EC35F0D3
:105A900018EC54F0FF0E58EC35F01AEC35F04A0EC5
:105AA00026EC35F0BF0E3FEC35F00B0E475CD8B45A
:105AB000A0EF2DF0000E58EC35F048EC51F0000E40
:105AC00058EC35F0F8EC51F0000E58EC35F0F8ECED
:105AD00051F0000E58EC35F088EC54F058EC52F0D0
:105AE000000E58EC35F088EC51F0000E58EC35F013
:105AF000A8EC51F0000E58EC35F0C8EC51F0000E57
:105B000058EC35F068EC52F0000E58EC35F01DEC16
:105B100035F0400E26EC35F0BF0E3FEC35F078EC5A
:105B200052F0000E58EC35F088EC51F0000E58ECB5
:105B300035F058EC52F0000E58EC35F0E4EF2DF053
:105B4000FF0E58EC35F0E8EC52F0FF0E58EC35F053
:105B500098EC53F0FF0E58EC35F098EC53F0FF0E34
:105B600058EC35F098EC54F0F8EC53F0FF0E58EC8C
:105B700035F028EC53F0FF0E58EC35F048EC53F0BC
:105B8000FF0E58EC35F068EC53F0FF0E58EC35F092
:105B900008EC54F0FF0E58EC35F01DEC35F0400EDB
:105BA00026EC35F0BF0E3FEC35F018EC54F0FF0E4C
:105BB00058EC35F028EC53F0FF0E58EC35F0F8ECCB
:105BC00053F0FF0E58EC35F049EC39F080B8FCEF9B
:105BD0002DF0070E585CD8B4F1EF2DF0582AFEEFE7
:105BE0002DF0586A3EB8FEEF2DF0010E446E42ECE7
:105BF00036F03E88FEEF2DF03E98586A42EF01F0F5
:105C00001AEC35F0460E26EC35F0B90E3FEC35F0C7
:105C1000000E475CD8B441EF2EF0010E475CD8B4BB
:105C200049EF2EF0020E475CD8B451EF2EF0030E70
:105C3000475CD8B459EF2EF0040E475CD8B461EF3E
:105C40002EF0050E475CD8B469EF2EF0060E475CC7
:105C5000D8B471EF2EF0070E475CD8B479EF2EF070
:105C6000080E475CD8B481EF2EF0090E475CD8B41B
:105C700089EF2EF00A0E475CD8B491EF2EF0EBEFCF
:105C80002EF0B5EC48F05DEC40F0F6EC40F07EEF25
:105C90002FF00EEC49F05DEC40F0F6EC40F07EEFBA
:105CA0002FF067EC49F05DEC40F0F6EC40F07EEF51
:105CB0002FF0C0EC49F05DEC40F0F6EC40F07EEFE8
:105CC0002FF019EC4AF05DEC40F0F6EC40F07EEF7E
:105CD0002FF072EC4AF05DEC40F0F6EC40F07EEF15
:105CE0002FF01BEC4BF05DEC40F0F6EC40F07EEF5B
:105CF0002FF0A9EC4BF05DEC40F0F6EC40F07EEFBD
:105D00002FF018EC4CF05DEC40F0F6EC40F07EEF3C
:105D10002FF0A1EC4CF05DEC40F0F6EC40F07EEFA3
:105D20002FF0000E58EC35F028EC52F0000E58EC35
:105D300035F078EC52F0000E58EC35F0B8EC51F03C
:105D4000000E58EC35F088EC51F0000E58EC35F0B0
:105D500058EC52F0000E58EC35F088EC54F068EC3A
:105D600052F0000E58EC35F088EC51F0000E58EC73
:105D700035F078EC52F0000E58EC35F01DEC35F0B3
:105D8000400E26EC35F0B90E3FEC35F0000E58EC25
:105D900035F0000E58EC35F0A8EC52F0000E58EC3F
:105DA00035F058EC52F0000E58EC35F0C8EC51F0DC
:105DB000000E58EC35F078EC52F0000E58EC35F04F
:105DC00088EC51F0000E58EC35F05DEC40F0F6EC4C
:105DD00040F07EEF2FF048EC51F0000E58EC35F01B
:105DE000F8EC51F0000E58EC35F0F8EC51F0000EE4
:105DF00058EC35F088EC54F058EC52F0000E58ECAA
:105E000035F088EC51F0000E58EC35F0A8EC51F06C
:105E1000000E58EC35F0C8EC51F0000E58EC35F09F
:105E200068EC52F0000E58EC35F078EC52F01DECB6
:105E300035F0400E26EC35F0B90E3FEC35F0000E93
:105E400058EC35F088EC51F0000E58EC35F058EC79
:105E500052F0000E58EC35F088EC54F0A8EC52F0FB
:105E6000000E58EC35F058EC52F0000E58EC35F0BE
:105E7000C8EC51F0000E58EC35F078EC52F0000E02
:105E800058EC35F088EC51F0000E58EC35F05DEC34
:105E900040F080B87CEF2FF0070E585CD8B454EF78
:105EA0002FF0582A7EEF2FF0586A3EB87EEF2FF081
:105EB0003FAC75EF2FF042EC36F020EC55F033ECB0
:105EC00055F046EC55F059EC55F06CEC55F07FEC84
:105ED00055F092EC55F0A5EC55F0B8EC55F0CBEC44
:105EE00055F0DEEC55F0F2EC55F0446A476A3F9C01
:105EF0003F903E8842EF01F03E98586A80BA42EFE8
:105F000001F0070E575CD8B489EF2FF0572A42EF03
:105F100001F0576A000E446E3E8A476A42EC36F042
:105F20003F9C42EF01F01AEC35F0410E26EC35F0C3
:105F3000B80E3FEC35F0700E58EC35F0100E58EC02
:105F400035F0100E58EC35F0100E58EC35F0000E10
:105F500058EC35F028EC52F0000E58EC35F078ECA7
:105F600052F0000E58EC35F0B8EC51F0000E58EC41
:105F700035F088EC51F0000E58EC35F058EC52F04A
:105F8000000E58EC35F088EC54F068EC52F0000E3E
:105F900058EC35F088EC51F0000E58EC35F078EC08
:105FA00052F0000E58EC35F078EC52F01DEC35F064
:105FB000400E26EC35F0B80E3FEC35F0000E58ECF4
:105FC00035F0C8EC51F0000E58EC35F018EC52F0FA
:105FD000000E58EC35F0A8EC51F0000E58EC35F0FE
:105FE000082A2C0E085CD8B4FBEF2FF0100E58ECEA
:105FF00035F0F0EF2FF0086A700E58EC35F034EC05
:1060000045F01AEC35F0460E26EC35F0BF0E3FECAD
:1060100035F068EC52F0000E58EC35F028EC52F0F8
:10602000000E58EC35F098EC51F0000E58EC35F0BD
:1060300078EC52F0000E58EC35F0A8EC52F0000E5F
:1060400058EC35F048EC51F0000E58EC35F058ECB7
:1060500052F0000E58EC35F088EC51F0000E58EC80
:1060600035F088EC54F098EC52F01DEC35F0400E11
:1060700026EC35F0BF0E3FEC35F0000E58EC35F055
:1060800088EC51F0000E58EC35F058EC52F0000E50
:1060900058EC35F068EC52F0000E58EC35F0C8ECD6
:1060A00051F0000E58EC35F028EC52F0000E58EC90
:1060B00035F018EC52F0000E58EC35F088EC54F046
:1060C000000E58EC35F088EC4EF0000E58EC35F030
:1060D000000E58EC35F0400E58EC35F0000E58EC40
:1060E00035F068EC4EF0000E58EC35F068EC4EF0F0
:1060F000000E58EC35F01AEC35F0400E26EC35F079
:10610000B90E3FEC35F04DBEBFEF30F0000E485CED
:10611000D8A4BFEF30F0FF0E58EC35F028EC53F068
:10612000FF0E58EC35F0F8EC53F0FF0E58EC35F05C
:10613000F8EC53F0FF0E58EC35F0C8EC53F0FF0EBE
:1061400058EC35F0F8EC53F0FF0E58EC35F098ECC5
:1061500054F058EC53F0FF0E58EC35F0C8EC53F007
:10616000FF0E58EC35F098EC53F0FF0E58EC35F07C
:1061700018EC53F0FF0E58EC35F0F1EF30F0000E54
:1061800058EC35F088EC51F0000E58EC35F058EC36
:1061900052F0000E58EC35F058EC52F0000E58EC6E
:1061A00035F028EC52F0000E58EC35F058EC52F077
:1061B000000E58EC35F088EC54F0B8EC51F0000EBD
:1061C00058EC35F028EC52F0000E58EC35F0F8ECB5
:1061D00051F0000E58EC35F078EC51F0000E58EC10
:1061E00035F01AEC35F0430E26EC35F0BA0E3FECE4
:1061F00035F01E0E58EC35F0100E58EC35F0100E40
:1062000058EC35F0100E58EC35F0100E58EC35F017
:106210001AEC35F0400E26EC35F0BB0E3FEC35F0B5
:106220004DBE47EF31F0010E485CD8A447EF31F086
:10623000FF0E58EC35F018EC54F0FF0E58EC35F02A
:1062400058EC54F0FF0E58EC35F098EC54F0C8ECD4
:1062500053F0FF0E58EC35F028EC54F0FF0E58ECDC
:1062600035F018EC54F0FF0E58EC35F0D8EC53F044
:10627000FF0E58EC35F028EC54F0FF0E58EC35F0DA
:1062800018EC54F0FF0E58EC35F074EF31F0000EBE
:1062900058EC35F078EC52F0000E58EC35F0B8ECD4
:1062A00052F0000E58EC35F088EC54F028EC52F027
:1062B000000E58EC35F088EC52F0000E58EC35F03A
:1062C00078EC52F0000E58EC35F038EC52F0000E3D
:1062D00058EC35F088EC52F0000E58EC35F078ECC4
:1062E00052F0000E58EC35F01AEC35F0430E26EC67
:1062F00035F0BC0E3FEC35F01E0E58EC35F0100EAC
:1063000058EC35F0100E58EC35F0100E58EC35F016
:10631000100E58EC35F01AEC35F0400E26EC35F046
:10632000BD0E3FEC35F04DBECFEF31F0020E485CB4
:10633000D8A4CFEF31F0FF0E58EC35F008EC54F054
:10634000FF0E58EC35F028EC53F0FF0E58EC35F00A
:1063500098EC53F0FF0E58EC35F028EC53F0FF0E9C
:1063600058EC35F008EC53F0FF0E58EC35F018EC13
:1063700054F0FF0E58EC35F098EC54F028EC54F043
:10638000FF0E58EC35F008EC54F0FF0E58EC35F0E9
:10639000F8EC52F0FF0E58EC35F001EF32F0000E41
:1063A00058EC35F068EC52F0000E58EC35F088EC03
:1063B00051F0000E58EC35F0F8EC51F0000E58ECAE
:1063C00035F088EC51F0000E58EC35F068EC51F0E7
:1063D000000E58EC35F078EC52F0000E58EC35F029
:1063E00088EC54F088EC52F0000E58EC35F068EC74
:1063F00052F0000E58EC35F058EC51F0000E58EC0D
:1064000035F01AEC35F0430E26EC35F0BE0E3FECBD
:1064100035F01E0E58EC35F0100E58EC35F0100E1D
:1064200058EC35F0100E58EC35F0100E58EC35F0F5
:106430004DBE56EF32F080B036EF32F0070E565CAC
:10644000D8B426EF32F0562A38EF32F0566A3EB012
:1064500038EF32F0020E485CD8B432EF32F0482AFE
:1064600033EF32F0486A3E8038EF32F03E90566AA1
:1064700084B654EF32F0070E555CD8B443EF32F0D7
:10648000552A56EF32F0556A3EBC56EF32F0000EF8
:10649000485CD8B44FEF32F0480651EF32F0020EAC
:1064A000486E3E8C56EF32F03E9C556A4DBE70EF02
:1064B00032F080B86EEF32F0070E585CD8B464EF5B
:1064C00032F0582A70EF32F0586A3EB870EF32F06E
:1064D0004D8E4D504E6E3E8870EF32F03E98586AA9
:1064E0004DAE8AEF32F080BA88EF32F0070E575C7B
:1064F000D8B47EEF32F0572A8AEF32F0576A3EBAAC
:106500008AEF32F04D9E4D504E6E3E8A8AEF32F049
:106510003E9A576A4DAEA6EF32F080B8A4EF32F043
:10652000070E585CD8B498EF32F0582AA6EF32F034
:10653000586A3EB8A6EF32F04E504D6E4D9E42EC7A
:1065400036F03E88A6EF32F03E98586A4DAE01EF25
:1065500033F080B0D3EF32F0070E565CD8B4B4EF0E
:1065600032F0562AD5EF32F0566A3EB0D5EF32F00F
:10657000000E485CD8B4C9EF32F0010E485CD8B4C4
:10658000CCEF32F0020E485CD8B4CFEF32F0D0EF4F
:1065900032F04E70D0EF32F04E72D0EF32F04E74D7
:1065A0003E80D5EF32F03E90566A84B6FFEF32F06F
:1065B000070E555CD8B4E0EF32F0552A01EF33F006
:1065C000556A3EBC01EF33F0000E485CD8B4F5EFDD
:1065D00032F0010E485CD8B4F8EF32F0020E485C9D
:1065E000D8B4FBEF32F0FCEF32F04E70FCEF32F03B
:1065F0004E72FCEF32F04E743E8C01EF33F03E9C55
:10660000556A1AEC35F04A0E26EC35F0BA0E3FEC1E
:1066100035F0000E485CD8A446EF33F04DAE46EF9F
:1066200033F04EA02DEF33F0FF0E58EC35F058EC60
:1066300053F0FF0E58EC35F0C8EC53F0FF0E58EC59
:1066400035F098EC53F0FF0E58EC35F018EC53F0A1
:10665000FF0E58EC35F079EF33F0FF0E58EC35F0C3
:1066600038EC53F0FF0E58EC35F0F8EC53F0FF0E19
:1066700058EC35F028EC53F0FF0E58EC35F028ECD0
:1066800053F0FF0E58EC35F079EF33F04EA062EF87
:1066900033F0000E58EC35F0B8EC51F0000E58EC29
:1066A00035F028EC52F0000E58EC35F0F8EC51F0D3
:1066B000000E58EC35F078EC51F0000E58EC35F047
:1066C00079EF33F0000E58EC35F098EC51F0000EF5
:1066D00058EC35F058EC52F0000E58EC35F088ECE0
:1066E00051F0000E58EC35F088EC51F0000E58ECEB
:1066F00035F01AEC35F04A0E26EC35F0BC0E3FECC6
:1067000035F0010E485CD8A400EF34F04DAE00EF38
:1067100034F04EA2C6EF33F0FF0E58EC35F068ECC3
:1067200053F0FF0E58EC35F0B8EC53F0FF0E58EC78
:1067300035F018EC54F0FF0E58EC35F028EC53F01F
:10674000FF0E58EC35F0F8EC53F0FF0E58EC35F036
:1067500098EC53F0FF0E58EC35F0C8EC53F0FF0EF8
:1067600058EC35F008EC53F0FF0E58EC35F088EC9F
:1067700053F01DEC35F0400E26EC35F0BC0E3FEC2E
:1067800035F0FF0E58EC35F075EF34F0FF0E58EC95
:1067900035F038EC53F0FF0E58EC35F0F8EC53F0D0
:1067A000FF0E58EC35F028EC53F0FF0E58EC35F0A6
:1067B00028EC53F0FF0E58EC35F088EC54F0000E46
:1067C00058EC35F088EC54F0000E58EC35F088ECBD
:1067D00054F0000E58EC35F088EC54F0000E58ECF4
:1067E00035F088EC54F01DEC35F0400E26EC35F019
:1067F000BC0E3FEC35F0000E58EC35F075EF34F080
:106800004EA23DEF34F0000E58EC35F0C8EC51F0DC
:10681000000E58EC35F018EC52F0000E58EC35F044
:1068200078EC52F0000E58EC35F088EC51F0000E88
:1068300058EC35F058EC52F0000E58EC35F0F8EC0E
:1068400051F0000E58EC35F028EC52F0000E58ECE8
:1068500035F068EC51F0000E58EC35F0E8EC51F0F2
:106860001DEC35F0400E26EC35F0BC0E3FEC35F05B
:10687000000E58EC35F075EF34F0000E58EC35F0A2
:1068800098EC51F0000E58EC35F058EC52F0000E38
:1068900058EC35F088EC51F0000E58EC35F088ECEF
:1068A00051F0000E58EC35F088EC54F0000E58EC26
:1068B00035F088EC54F0000E58EC35F088EC54F0CC
:1068C000000E58EC35F088EC54F0000E58EC35F022
:1068D00088EC54F01DEC35F0400E26EC35F0BC0E83
:1068E0003FEC35F0000E58EC35F01AEC35F04A0E5E
:1068F00026EC35F0BE0E3FEC35F0020E485CD8A415
:10690000CEEF34F04DAECEEF34F04EA4ABEF34F01A
:10691000FF0E58EC35F0E8EC52F0FF0E58EC35F075
:1069200028EC54F0FF0E58EC35F018EC54F0FF0E44
:1069300058EC35F0C8EC53F0FF0E58EC35F088EC0D
:1069400054F0000E58EC35F088EC54F0000E58EC82
:1069500035F015EF35F0FF0E58EC35F0A8EC53F09C
:10696000FF0E58EC35F0E8EC52F0FF0E58EC35F025
:10697000B8EC53F0FF0E58EC35F028EC54F0FF0E55
:1069800058EC35F0E8EC52F0FF0E58EC35F098EC8E
:1069900053F0FF0E58EC35F015EF35F04EA4F4EF40
:1069A00034F0000E58EC35F048EC51F0000E58EC85
:1069B00035F088EC52F0000E58EC35F078EC52F0DF
:1069C000000E58EC35F028EC52F0000E58EC35F083
:1069D00088EC54F0000E58EC35F088EC54F0000EC2
:1069E00058EC35F015EF35F0000E58EC35F008ECAA
:1069F00052F0000E58EC35F048EC51F0000E58EC17
:106A000035F018EC52F0000E58EC35F088EC52F0EE
:106A1000000E58EC35F048EC51F0000E58EC35F013
:106A2000F8EC51F0000E58EC35F04DAE49EC39F071
:106A300042EF01F08C888B9E12008C988B8E120096
:106A40008C888B8E12008C988B9E1200016E1FEC2E
:106A500036F001508A6E8C9C8C9E000000008C8A5F
:106A60000000000000000000000000000000000026
:106A70008C9A000000000000000000001200026E6E
:106A80001FEC36F002508A6E8C9C8C9E0000000039
:106A90008C8A0000000000000000000000000000E0
:106AA00000008C9A000000000000000000001200AE
:106AB000006E1FEC36F03FBE74EC35F000508A6E6D
:106AC0008C9C8C8E000000008C8A0000000000006E
:106AD000000000000000000000008C9A0000000090
:106AE0000000000000001200000E525CD8B499EFC4
:106AF00035F0010E525CD8B4B2EF35F0020E525CA4
:106B0000D8B4C9EF35F0030E525CD8B4DEEF35F0DF
:106B1000040E525CD8B4F1EF35F0050E525CD8B4D7
:106B200002EF36F0060E525CD8B411EF36F01EEFCD
:106B300036F051B0A7EF35F000420042004200426B
:106B4000004200420042010E00161EEF36F00046E1
:106B5000004600460046004600460046800E0016ED
:106B60001EEF36F051B0BFEF35F000420042004258
:106B7000004200420042030E00161EEF36F00046AF
:106B800000460046004600460046C00E00161EEFB6
:106B900036F051B0D5EF35F00042004200420042DD
:106BA0000042070E00161EEF36F000460046004673
:106BB00000460046E00E00161EEF36F051B0E9EF39
:106BC00035F000420042004200420F0E00161EEF58
:106BD00036F00046004600460046F00E00161EEF56
:106BE00036F051B0FBEF35F00042004200421F0E7C
:106BF00000161EEF36F0004600460046F80E00165E
:106C00001EEF36F051B00BEF36F0004200423F0E5F
:106C100000161EEF36F000460046FC0E00161EEF72
:106C200036F051B019EF36F000427F0E00161EEF1D
:106C300036F00046FE0E00161EEF36F012000F0171
:106C4000FF0E936E00018C8C8C9E000000008C8ADD
:106C50000000000000000000000000000000000034
:106C60008C9A0000000000000000000000000000FE
:106C7000000081BE27EF36F08C9C0F01000E936E52
:106C80000001120020EC35F0400E26EC35F0B80E75
:106C90003FEC35F0000E58EC35F0012A800E015C17
:106CA000D8A44AEF36F0022A40EC35F0400E26EC2C
:106CB00035F0C00E025CD8A44AEF36F012008B808B
:106CC00000008B92ACEC42F08B82ACEC42F07CEC9E
:106CD00036F092EC36F0BCEC36F0D1EC36F0E6EC67
:106CE00036F0FBEC36F010EC37F025EC37F03AECF0
:106CF00037F04FEC37F012008B90000064EC37F067
:106D00008B9400008B8600008B960000000E386E7E
:106D10008FEC37F011503C6EA4EC37F08B948B96CF
:106D20008B8012008B9064EC37F08B9400008B8684
:106D300000008B960000010E386E8FEC37F0125079
:106D40003C6EA4EC37F08B948B968B8012008B906A
:106D500064EC37F08B9400008B8600008B9600006B
:106D6000010E386E8FEC37F0400E3C6EA4EC37F01D
:106D70008B948B968B8012008B9064EC37F08B9405
:106D800000008B8600008B960000020E386E8FECA0
:106D900037F013503C6EA4EC37F08B948B968B80BD
:106DA00012008B9064EC37F08B9400008B8600000F
:106DB0008B960000030E386E8FEC37F014503C6E4B
:106DC000A4EC37F08B948B968B8012008B9064EC44
:106DD00037F08B9400008B8600008B960000040E29
:106DE000386E8FEC37F015503C6EA4EC37F08B9476
:106DF0008B968B8012008B9064EC37F08B940000A4
:106E00008B8600008B960000050E386E8FEC37F0F5
:106E100016503C6EA4EC37F08B948B968B8012004E
:106E20008B9064EC37F08B9400008B8600008B967F
:106E30000000060E386E8FEC37F017503C6EA4EC55
:106E400037F08B948B968B8012008B9064EC37F02C
:106E50008B9400008B8600008B960000070E386E26
:106E60008FEC37F018503C6EA4EC37F08B948B9677
:106E70008B8012008B9064EC37F08B9400008B8633
:106E800000008B960000080E386E8FEC37F019501A
:106E90003C6EA4EC37F08B948B968B8012008B9019
:106EA00064EC37F08B9400008B8600008B9600001A
:106EB000090E386E8FEC37F01A503C6EA4EC37F0A8
:106EC0008B948B968B8012008B9400008B86000035
:106ED0008B9600008B9400008B8600008B96000040
:106EE0008B8400008B8600008B9600008B94000042
:106EF0008B8600008B9600008B9400008B86000030
:106F00008B9600008B9400008B8600008B9600000F
:106F10008B9400008B8600008B960000120038BE18
:106F200095EF37F08B9497EF37F08B8400008B86CA
:106F300000008B960000392A3846080E395CD8A428
:106F40008FEF37F0396A12003CBEAAEF37F08B940E
:106F5000ACEF37F08B8400008B8600008B9600002E
:106F60003A2A3C46080E3A5CD8A4A4EF37F03A6AB5
:106F700012008B9064EC37F08B9400008B8600003D
:106F80008B9600000A0E386E8FEC37F08B80000075
:106F9000000000008B9064EC37F08B8400008B863F
:106FA00000008B960000000000000000DCEC37F0D1
:106FB0008B948B968B8012008B8683A0E3EF37F047
:106FC0003B80E4EF37F03B903A2A8B96080E3A5C10
:106FD000D8B4EEEF37F03B46DCEF37F03A6A3D2AA3
:106FE000010E3D5CD8A4F9EF37F03B501B6EDCEF8F
:106FF00037F0020E3D5CD8A402EF38F03B501C6E17
:10700000DCEF37F0030E3D5CD8A40BEF38F03B50BB
:107010001D6EDCEF37F0040E3D5CD8A414EF38F0A1
:107020003B501E6EDCEF37F0050E3D5CD8A41DEF23
:1070300038F03B501F6EDCEF37F0060E3D5CD8A4F5
:1070400026EF38F03B50206EDCEF37F0070E3D5C4A
:10705000D8A42FEF38F03B50216EDCEF37F0080E4C
:107060003D5CD8A438EF38F03B50226EDCEF37F0AF
:10707000090E3D5CD8A441EF38F03B50236EDCEFA5
:1070800037F00A0E3D5CD8A44AEF38F03B50246E2E
:10709000DCEF37F00B0E3D5CD8A453EF38F03B50DB
:1070A000256EDCEF37F00C0E3D5CD8A45CEF38F0B9
:1070B0003B50266EDCEF37F00D0E3D5CD8A465EF3B
:1070C00038F03B50276EDCEF37F00E0E3D5CD8A455
:1070D0006EEF38F03B50286EDCEF37F00F0E3D5C62
:1070E000D8A477EF38F03B50296EDCEF37F0100E64
:1070F0003D5CD8A480EF38F03B502A6EDCEF37F0CF
:10710000110E3D5CD8A489EF38F03B502B6EDCEFBC
:1071100037F0120E3D5CD8A492EF38F03B502C6E45
:10712000DCEF37F0130E3D5CD8A49BEF38F03B50FA
:107130002D6EDCEF37F0140E3D5CD8A4A4EF38F0D0
:107140003B502E6EDCEF37F0150E3D5CD8A4ADEF52
:1071500038F03B502F6EDCEF37F0160E3D5CD8A4B4
:10716000B6EF38F03B50306EDCEF37F0170E3D5C79
:10717000D8A4BFEF38F03B50316EDCEF37F0180E7B
:107180003D5CD8A4C8EF38F03B50326EDCEF37F0EE
:10719000190E3D5CD8A4D1EF38F03B50336EDCEFD4
:1071A00037F01A0E3D5CD8A4DAEF38F03B50346E5D
:1071B000DCEF37F01B0E3D5CD8A4E3EF38F03B501A
:1071C000356EDCEF37F01C0E3D5CD8A4ECEF38F0E8
:1071D0003B50366EDCEF37F03B50376E3D6A1200A5
:1071E0001650BF0B616FA80E615DD8B428EF39F05F
:1071F000980E615DD8B42BEF39F0880E615DD8B47C
:107200002EEF39F0619F250E615DD8B431EF39F072
:10721000150E615DD8B434EF39F0050E615DD8B458
:1072200037EF39F0200E615DD8B43AEF39F0100E27
:10723000615DD8B43DEF39F0000E615DD8B440EF28
:1072400039F0300E615DD8B443EF39F046EF39F0D4
:10725000000E47EF39F0010E47EF39F0020E47EF0D
:1072600039F0030E47EF39F0040E47EF39F0050E01
:1072700047EF39F0060E47EF39F0070E47EF39F0C8
:10728000080E47EF39F0090E47EF39F00F0E5D6E2B
:10729000120080BA99EF39F0070E575CD8B454EF5A
:1072A00039F0572A9BEF39F0576A3EBA1200000EA8
:1072B000415CD8B497EF39F0010E415CD8B494EF3B
:1072C00039F0020E415CD8B472EF39F0030E415C24
:1072D000D8B47BEF39F0040E415CD8B484EF39F0B8
:1072E0008DEF39F0466A44A0476A4DAE486A51AE08
:1072F000496A94EF39F0496A43A0466A44A0476A54
:107300004DAE486A94EF39F043A0466A476A4DAEE5
:10731000486A51AE496A94EF39F043A0466A44A0E6
:10732000476A486A51AE496A42EC36F0416A3E8A81
:1073300012003E9A576A12005E0E295CD8B4E4EF40
:1073400039F05D0E295CD8B4E4EF39F0440E295CC5
:10735000D8B4EAEF39F0450E295CD8B4EAEF39F039
:107360003E0E295CD8B4F0EF39F03F0E295CD8B45A
:10737000F0EF39F0220E295CD8B4F6EF39F0230E85
:10738000295CD8B4F6EF39F01F0E295CD8B4FCEFB5
:1073900039F0200E295CD8B4FCEF39F0110E295CCD
:1073A000D8B402EF3AF0120E295CD8B402EF3AF0EA
:1073B000100E295CD8B408EF3AF00F0E295CD8B44F
:1073C00008EF3AF00EEF3AF0010E626F010E636FB4
:1073D00012EF3AF0020E626F010E636F12EF3AF095
:1073E000030E626F010E636F12EF3AF0040E626FCC
:1073F000010E636F12EF3AF0050E626F010E636FBC
:1074000012EF3AF0060E626F020E636F12EF3AF05F
:10741000070E626F020E636F12EF3AF0FE0E626F9C
:10742000030E636F5FA212006351645DD8A41BEF6B
:107430003AF02DEF3AF0010E635DD8B427EF3AF041
:10744000020E635DD8B42AEF3AF02DEF3AF01292B3
:107450002BEF3AF0128292EC36F06351646F120017
:10746000000E405CD8A459EF3AF0A8EC51F0000EA1
:1074700058EC35F018EC52F0000E58EC35F078EC82
:1074800051F0000E58EC35F088EC54F0000E58EC3A
:1074900035F088EC54F0000E58EC35F088EC54F0E0
:1074A000000E58EC35F088EC54F0000E58EC35F036
:1074B0001200010E405CD8A482EF3AF088EC51F043
:1074C000000E58EC35F008EC52F0000E58EC35F098
:1074D00038EC52F0000E58EC35F0B8EC51F0000EDC
:1074E00058EC35F088EC54F0000E58EC35F088EC90
:1074F00054F0000E58EC35F088EC54F0000E58ECC7
:1075000035F01200020E405CD8A4ABEF3AF0C8ECA4
:1075100051F0000E58EC35F018EC52F0000E58EC1B
:1075200035F078EC52F0000E58EC35F088EC54F061
:10753000000E58EC35F088EC54F0000E58EC35F0A5
:1075400088EC54F0000E58EC35F088EC54F0000E46
:1075500058EC35F01200030E405CD8A4D4EF3AF09A
:1075600068EC51F0000E58EC35F088EC54F0000E49
:1075700058EC35F068EC52F0000E58EC35F078EC31
:1075800052F0000E58EC35F048EC51F0000E58EC7B
:1075900035F088EC54F0000E58EC35F088EC54F0DF
:1075A000000E58EC35F01200040E405CD8A4FDEF3C
:1075B0003AF088EC52F0000E58EC35F088EC54F0BC
:1075C000000E58EC35F078EC51F0000E58EC35F028
:1075D00048EC51F0000E58EC35F078EC52F0000E0B
:1075E00058EC35F048EC51F0000E58EC35F088ECD2
:1075F00054F0000E58EC35F01200050E405CD8A493
:1076000026EF3BF058EC52F0000E58EC35F088ECC9
:1076100054F0000E58EC35F088EC51F0000E58ECA8
:1076200035F058EC52F0000E58EC35F058EC52F0B2
:10763000000E58EC35F088EC54F0000E58EC35F0A4
:1076400088EC54F0000E58EC35F01200060E405C49
:10765000D8A44FEF3BF018EC52F0000E58EC35F088
:1076600098EC52F0000E58EC35F088EC54F0000E17
:1076700058EC35F088EC51F0000E58EC35F058EC31
:1076800052F0000E58EC35F058EC52F0000E58EC69
:1076900035F088EC54F0000E58EC35F01200070E6F
:1076A000405CD8A478EF3BF058EC52F0000E58EC58
:1076B00035F068EC51F0000E58EC35F058EC51F014
:1076C000000E58EC35F0F8EC51F0000E58EC35F0A7
:1076D00088EC54F0000E58EC35F088EC54F0000EB5
:1076E00058EC35F088EC54F0000E58EC35F01200F0
:1076F000080E405CD8A4A1EF3BF0F8EC4EF0000E71
:1077000058EC35F0C8EC4EF0000E58EC35F0E8ECD3
:1077100051F0000E58EC35F0B8EC51F0000E58EC7A
:1077200035F0D8EC52F0000E58EC35F088EC54F0FF
:10773000000E58EC35F088EC54F0000E58EC35F0A3
:107740001200090E405CD8A4CAEF3BF048EC51F09F
:10775000000E58EC35F088EC52F0000E58EC35F085
:1077600078EC51F0000E58EC35F0C8EC51F0000EFA
:1077700058EC35F028EC52F0000E58EC35F088EC5F
:1077800054F0000E58EC35F088EC54F0000E58EC34
:1077900035F012000A0E405CD8A4F3EF3BF098ECF1
:1077A00052F0000E58EC35F0F8EC51F0000E58ECA9
:1077B00035F058EC52F0000E58EC35F068EC51F012
:1077C000000E58EC35F0E8EC51F0000E58EC35F0B6
:1077D00088EC54F0000E58EC35F088EC54F0000EB4
:1077E00058EC35F012000B0E405CD8A4D5EF3CF0FD
:1077F00078EC52F0000E58EC35F0B8EC52F0000E78
:1078000058EC35F088EC54F0000E58EC35F015507B
:10781000070B406E000E405CD8A424EF3CF058ECFF
:1078200052F0000E58EC35F0B8EC52F0000E58EC67
:1078300035F038EC52F0000E58EC35F068EC4EF0B4
:10784000000E58EC35F01200010E405CD8A43EEF5B
:107850003CF058EC52F0000E58EC35F0B8EC52F019
:10786000000E58EC35F038EC52F0000E58EC35F0C4
:1078700078EC4EF0000E58EC35F01200020E405C31
:10788000D8A458EF3CF058EC52F0000E58EC35F00C
:10789000B8EC52F0000E58EC35F038EC52F0000E17
:1078A00058EC35F088EC4EF0000E58EC35F0120034
:1078B000030E405CD8A472EF3CF088EC52F0000E4E
:1078C00058EC35F068EC52F0000E58EC35F058ECFE
:1078D00051F0000E58EC35F088EC54F0000E58ECE6
:1078E00035F01200040E405CD8A48CEF3CF058EC4C
:1078F00052F0000E58EC35F0B8EC52F0000E58EC97
:1079000035F038EC52F0000E58EC35F0A8EC4EF0A3
:10791000000E58EC35F01200050E405CD8A4A6EF1E
:107920003CF058EC52F0000E58EC35F0B8EC52F048
:10793000000E58EC35F038EC52F0000E58EC35F0F3
:10794000B8EC4EF0000E58EC35F01200060E405C1C
:10795000D8A4C0EF3CF058EC52F0000E58EC35F0D3
:10796000B8EC52F0000E58EC35F038EC52F0000E46
:1079700058EC35F0C8EC4EF0000E58EC35F0120023
:1079800058EC52F0000E58EC35F0B8EC52F0000E06
:1079900058EC35F038EC52F0000E58EC35F0D8ECDD
:1079A0004EF0000E58EC35F012000C0E405CD8A4DE
:1079B000FEEF3CF098EC52F0000E58EC35F078EC0D
:1079C00051F0000E58EC35F078EC51F0000E58EC08
:1079D00035F088EC54F0000E58EC35F088EC54F09B
:1079E000000E58EC35F088EC54F0000E58EC35F0F1
:1079F00088EC54F0000E58EC35F012000D0E405C8F
:107A0000D8A427EF3DF0B8EC51F0000E58EC35F05B
:107A100058EC52F0000E58EC35F008EC52F0000E25
:107A200058EC35F068EC51F0000E58EC35F0E8EC0D
:107A300051F0000E58EC35F088EC54F0000E58EC84
:107A400035F088EC54F0000E58EC35F0120058EC8C
:107A500052F0000E58EC35F088EC51F0000E58EC66
:107A600035F068EC52F0000E58EC35F088EC51F02F
:107A7000000E58EC35F058EC52F0000E58EC35F092
:107A800098EC52F0000E58EC35F088EC51F0000EF6
:107A900058EC35F0120080B067EF3DF0070E565CF1
:107AA000D8B456EF3DF0562A69EF3DF0566A3EB025
:107AB00069EF3DF0000E4A5CD8A463EF3DF0080E7C
:107AC0004A6E64EF3DF04A063E8069EF3DF03E901D
:107AD000566A84B685EF3DF0070E555CD8B474EF56
:107AE0003DF0552A87EF3DF0556A3EBC87EF3DF0EB
:107AF000080E4A5CD8A481EF3DF0000E4A6E82EF7A
:107B00003DF04A2A3E8C87EF3DF03E9C556A1200BC
:107B100080B0A4EF3DF0070E565CD8B493EF3DF073
:107B2000562AA6EF3DF0566A3EB0A6EF3DF0010E94
:107B30004A5CD8A4A0EF3DF0080E4A6EA1EF3DF0DC
:107B40004A063E80A6EF3DF03E90566A84B6C2EFEC
:107B50003DF0070E555CD8B4B1EF3DF0552AC4EFA7
:107B60003DF0556A3EBCC4EF3DF0080E4A5CD8A417
:107B7000BEEF3DF0010E4A6EBFEF3DF04A2A3E8C4B
:107B8000C4EF3DF03E9C556A1200080E4A5CD8B422
:107B9000DCEF3FF03FB40BEF3EF080B8E0EF3DF09C
:107BA000070E585CD8B4D8EF3DF0582AE2EF3DF00C
:107BB000586A3EB89EEF3EF03F843E880BEF3EF0A1
:107BC0003E98586A1AEC35F04D0E26EC35F0BE0E94
:107BD0003FEC35F0000E58EC35F088EC54F0000E18
:107BE00058EC35F088EC54F088EC54F0000E58EC6A
:107BF00035F088EC54F0000E58EC35F088EC54F079
:107C0000000E58EC35F088EC54F0000E58EC35F0CE
:107C10004B50406E12001AEC35F04D0E26EC35F04C
:107C2000BE0E3FEC35F0000E4A5CD8B438EF3EF0A3
:107C3000010E4A5CD8B43DEF3EF0020E4A5CD8B467
:107C400042EF3EF0030E4A5CD8B447EF3EF0040E1C
:107C50004A5CD8B44CEF3EF0050E4A5CD8B451EF04
:107C60003EF0060E4A5CD8B456EF3EF05BEF3EF0B5
:107C70004CAE60EF3EF080EF3EF04CAC60EF3EF07B
:107C800080EF3EF04CAA60EF3EF080EF3EF04CA853
:107C900060EF3EF080EF3EF04CA660EF3EF080EFEC
:107CA0003EF04CA460EF3EF080EF3EF04CA260EF5F
:107CB0003EF080EF3EF04CA060EF3EF080EF3EF0F3
:107CC000000E58EC35F078EC4EF0000E58EC35F024
:107CD00088EC54F028EC52F0000E58EC35F058ECDB
:107CE00052F0000E58EC35F088EC54F0FF0E58ECD2
:107CF00035F008EC4FF0FF0E58EC35F09EEF3EF0FB
:107D0000FF0E58EC35F018EC4FF0FF0E58EC35F044
:107D100088EC54F028EC52F0000E58EC35F058EC9A
:107D200052F0000E58EC35F088EC54F0000E58EC90
:107D300035F068EC4EF0000E58EC35F04B50406ECC
:107D40003FA4120080BAB7EF3EF0070E575CD8B4DC
:107D5000ADEF3EF0572AB9EF3EF0576A3EBAB9EFA1
:107D60003EF03F944B50406E4C6E3E8A12003E9A5D
:107D7000576A80B83BEF3FF0070E585CD8B4C4EFA9
:107D80003EF0582A3DEF3FF0586A3EB83DEF3FF0D5
:107D9000000E4A5CD8B4EDEF3EF0010E4A5CD8B458
:107DA000F6EF3EF0020E4A5CD8B4FFEF3EF0030E51
:107DB0004A5CD8B408EF3FF0040E4A5CD8B411EF27
:107DC0003FF0050E4A5CD8B41AEF3FF0060E4A5C4D
:107DD000D8B423EF3FF02CEF3FF04CAEF3EF3EF082
:107DE0004B8E35EF3FF04B9E35EF3FF04CACFCEF48
:107DF0003EF04B8C35EF3FF04B9C35EF3FF04CAAFB
:107E000005EF3FF04B8A35EF3FF04B9A35EF3FF0EF
:107E10004CA80EEF3FF04B8835EF3FF04B9835EF15
:107E20003FF04CA617EF3FF04B8635EF3FF04B96F7
:107E300035EF3FF04CA420EF3FF04B8435EF3FF09F
:107E40004B9435EF3FF04CA229EF3FF04B8235EFDA
:107E50003FF04B9235EF3FF04CA032EF3FF04B80BC
:107E600035EF3FF04B9035EF3FF03F944B50406E75
:107E70003E883DEF3FF03E98586A80B08AEF3FF071
:107E8000070E565CD8B448EF3FF0562A8CEF3FF00F
:107E9000566A3EB08CEF3FF0000E4A5CD8B471EFEA
:107EA0003FF0010E4A5CD8B474EF3FF0020E4A5C1A
:107EB000D8B477EF3FF0030E4A5CD8B47AEF3FF0C6
:107EC000040E4A5CD8B47DEF3FF0050E4A5CD8B48E
:107ED00080EF3FF0060E4A5CD8B483EF3FF086EFA8
:107EE0003FF04C7E87EF3FF04C7C87EF3FF04C7AC1
:107EF00087EF3FF04C7887EF3FF04C7687EF3FF00D
:107F00004C7487EF3FF04C7287EF3FF04C703E802F
:107F10008CEF3FF03E90566A84B6D9EF3FF0070EE3
:107F2000555CD8B497EF3FF0552ADCEF3FF0556A27
:107F30003EBCDBEF3FF0000E4A5CD8B4C0EF3FF030
:107F4000010E4A5CD8B4C3EF3FF0020E4A5CD8B4CD
:107F5000C6EF3FF0030E4A5CD8B4C9EF3FF0040E01
:107F60004A5CD8B4CCEF3FF0050E4A5CD8B4CFEFF2
:107F70003FF0060E4A5CD8B4D2EF3FF0D5EF3FF0A9
:107F80004C7ED6EF3FF04C7CD6EF3FF04C7AD6EFEC
:107F90003FF04C78D6EF3FF04C76D6EF3FF04C7484
:107FA000D6EF3FF04C72D6EF3FF04C703E8CDBEFDB
:107FB0003FF03E9C556A120080B85AEF40F0070E21
:107FC000585CD8B4E7EF3FF0582A5CEF40F0586AAD
:107FD0003EB85CEF40F0000E465CD8B41EEF40F0B7
:107FE000010E465CD8B422EF40F0020E465CD8B4D5
:107FF00026EF40F0030E465CD8B42AEF40F0040EA2
:10800000465CD8B42EEF40F0050E465CD8B432EF93
:1080100040F0060E465CD8B43AEF40F0070E465CDE
:10802000D8B43EEF40F0080E465CD8B442EF40F0C2
:10803000090E465CD8B446EF40F012004B50116E6A
:1080400048EF40F04B50126E48EF40F04B50136E2B
:1080500048EF40F04B50146E48EF40F04B50156E17
:1080600048EF40F04B50166EF0EC38F05D505E6E0D
:1080700048EF40F04B50176E48EF40F04B50186EF1
:1080800048EF40F04B50196E48EF40F04B501A6EDD
:108090005FEC36F04B50406E3E88000E465CD8B424
:1080A00056EF40F0070E4A6E5CEF40F0050E4A6E48
:1080B0005CEF40F03E98586A12001AEC35F0670EFB
:1080C00026EC35F0BC0E3FEC35F03FBC7CEF40F0C9
:1080D000000E58EC35F0C8EC52F0000E58EC35F0BC
:1080E00088EC51F0000E58EC35F068EC52F0000EC0
:1080F00058EC35F08EEF40F0FF0E58EC35F068ECA0
:1081000054F0FF0E58EC35F028EC53F0FF0E58EC0D
:1081100035F008EC54F0FF0E58EC35F01DEC35F05E
:10812000440E26EC35F0BC0E3FEC35F03FBCADEF15
:1081300040F0FF0E58EC35F0B8EC53F0FF0E58EC61
:1081400035F098EC54F0FF0E58EC35F0C8EC53F0D5
:10815000FF0E58EC35F0BFEF40F0000E58EC35F054
:1081600018EC52F0000E58EC35F088EC54F0000E8C
:1081700058EC35F028EC52F0000E58EC35F080B099
:10818000D8EF40F0070E565CD8B4CAEF40F0562A3C
:10819000DAEF40F0566A3EB0DAEF40F03FBCD4EF81
:1081A00040F03F8CD5EF40F03F9C3E80DAEF40F04E
:1081B0003E90566A84B6F3EF40F0070E555CD8B493
:1081C000E5EF40F0552AF5EF40F0556A3EBCF5EF7B
:1081D00040F03FBCEFEF40F03F8CF0EF40F03F9CB1
:1081E0003E8CF5EF40F03E9C556A120080B877EF68
:1081F00041F0070E585CD8B401EF41F0582A79EFEE
:1082000041F0586A3EB879EF41F03FAC6FEF41F072
:1082100042EC36F0000E475CD8B443EF41F0010E5B
:10822000475CD8B447EF41F0020E475CD8B44BEF3F
:1082300041F0030E475CD8B44FEF41F0040E475CA9
:10824000D8B453EF41F0050E475CD8B457EF41F076
:10825000060E475CD8B45BEF41F0070E475CD8B41C
:108260005FEF41F0080E475CD8B463EF41F0090EB0
:10827000475CD8B467EF41F00A0E475CD8B46BEFA7
:1082800041F06FEF41F020EC55F06FEF41F033EC2F
:1082900055F06FEF41F046EC55F06FEF41F059ECBF
:1082A00055F06FEF41F06CEC55F06FEF41F07FEC63
:1082B00055F06FEF41F092EC55F06FEF41F0A5EC07
:1082C00055F06FEF41F0B8EC55F06FEF41F0CBECAB
:1082D00055F06FEF41F0DEEC55F0F2EC55F042EC6A
:1082E00036F0446A476A3F9C3E8842EF01F03E9870
:1082F000586A120083A29AEF41F03FB812004DB2C3
:108300008CEF41F01550380B406E180E406E155032
:10831000C70B156E94EF41F015503F0B406E1B0ECE
:10832000406E1550C00B156E405015125FEC36F0C4
:108330003F8812003F9812001550380B406E4042A3
:10834000404240424050070B406E1550F80B156EEE
:10835000405015121200106E000E105CD8A4C9EF28
:1083600041F005B8BAEF41F005BABEEF41F0C8ECF4
:108370004DF0120088EC54F0058C120005BCC5EFDE
:1083800041F0059CC8EC4DF01200059C88EC54F0BF
:108390001200010E105CD8A4D1EF41F0D8EC4DF0E2
:1083A0001200020E105CD8A4D9EF41F0E8EC4DF0B9
:1083B0001200030E105CD8A4E1EF41F0F8EC4DF090
:1083C0001200040E105CD8A4E9EF41F008EC4EF066
:1083D0001200050E105CD8A4F1EF41F018EC4EF03D
:1083E0001200060E105CD8A4F9EF41F028EC4EF014
:1083F0001200070E105CD8A401EF42F038EC4EF0EA
:108400001200080E105CD8A409EF42F048EC4EF0C0
:10841000120058EC4EF01200106E000E105CD8A442
:1084200015EF42F068EC4EF01200010E105CD8A47B
:108430001DEF42F078EC4EF01200020E105CD8A452
:1084400025EF42F088EC4EF01200030E105CD8A429
:108450002DEF42F098EC4EF01200040E105CD8A400
:1084600035EF42F0A8EC4EF01200050E105CD8A4D7
:108470003DEF42F0B8EC4EF01200060E105CD8A4AE
:1084800045EF42F0C8EC4EF01200070E105CD8A485
:108490004DEF42F0D8EC4EF01200080E105CD8A45C
:1084A00055EF42F0E8EC4EF01200F8EC4EF01200FE
:1084B000106E000E105CD8A461EF42F008EC4FF093
:1084C0001200010E105CD8A469EF42F018EC4FF0D6
:1084D0001200020E105CD8A471EF42F028EC4FF0AD
:1084E0001200030E105CD8A479EF42F038EC4FF084
:1084F0001200040E105CD8A481EF42F048EC4FF05B
:108500001200050E105CD8A489EF42F058EC4FF031
:108510001200060E105CD8A491EF42F068EC4FF008
:108520001200070E105CD8A499EF42F078EC4FF0DF
:108530001200080E105CD8A4A1EF42F088EC4FF0B6
:10854000120098EC4FF01200062A0A0E065CD8A41E
:10855000A4EF42F0066A1200062AFF0E065CD8A4B9
:10856000ACEF42F0066A072A640E075CD8A4ACEFB1
:1085700042F0066A076A1200062AFF0E065CD8A4BB
:10858000BCEF42F0066A072AFF0E075CD8A4BCEFD6
:1085900042F0066A076A12001AEC35F0400E26EC2B
:1085A00035F0BF0E3FEC35F078EC51F0000E58EC92
:1085B00035F048EC51F0000E58EC35F0C8EC51F0B5
:1085C000000E58EC35F0E8EC4EF0000E58EC35F0AB
:1085D000A8EC4EF0000E58EC35F078EC4EF0000EA2
:1085E00058EC35F0C8EC4EF088EC54F058EC52F0F2
:1085F000000E58EC35F088EC51F0000E58EC35F0D8
:1086000098EC52F01DEC35F0400E26EC35F0BF0E24
:108610003FEC35F0400E58EC35F0000E58EC35F0DC
:1086200078EC4EF0000E58EC35F0400E58EC35F07A
:10863000000E58EC35F068EC4EF0000E58EC35F0BA
:10864000400E036E7F0E046E1AEC35F0035026ECDC
:1086500035F0BC0E3FEC35F0010E58EC35F01DEC5A
:1086600035F0045026EC35F0BC0E3FEC35F0010E31
:1086700058EC35F0032A0406ACEC42F0800E035CA3
:10868000D8A424EF43F0BCEC42F0BCEC42F0BCECCC
:1086900042F0BCEC42F0BCEC42F0400E036E7F0EA8
:1086A000046E1AEC35F0035026EC35F0BC0E3FECAE
:1086B00035F0000E58EC35F01DEC35F0045026EC8A
:1086C00035F0BC0E3FEC35F0000E58EC35F0032AC7
:1086D0000406ACEC42F0800E035CD8A451EF43F0EA
:1086E0003F8EBCEC42F0BCEC42F0BCEC42F0BCEC87
:1086F00042F051801AEC35F04A0E26EC35F0BB0EF4
:108700003FEC35F0F8EC4FF0000E58EC35F0100E61
:1087100058EC35F0100E58EC35F0100E58EC35F0E2
:10872000100E58EC35F0100E58EC35F0000E58ECE9
:1087300035F078EC50F0000E58EC35F088EC54F041
:10874000000E58EC35F0E8EC4FF0000E58EC35F028
:1087500078EC50F0000E58EC35F008EC50F0000EBC
:1087600058EC35F028EC50F0000E58EC35F078EC71
:1087700050F0000E58EC35F01DEC35F0400E26ECB4
:1087800035F0BB0E3FEC35F0E8EC4FF0000E58EC46
:1087900035F0E8EC4FF0000E58EC35F0B8EC50F046
:1087A000000E58EC35F028EC50F0000E58EC35F087
:1087B00078EC50F0000E58EC35F008EC50F0000E5C
:1087C00058EC35F051901AEC35F0560E26EC35F099
:1087D000BC0E3FEC35F0A8EC4FF0000E58EC35F035
:1087E000E8EC50F0000E58EC35F0D8EC4FF0000EED
:1087F00058EC35F028EC50F0000E58EC35F088ECD1
:1088000050F0000E58EC35F088EC54F0000E58ECA7
:1088100035F058EC50F0000E58EC35F01DEC35F00A
:10882000400E26EC35F0BC0E3FEC35F0A8EC4FF0D6
:10883000000E58EC35F0B8EC4FF0000E58EC35F067
:1088400088EC50F0000E58EC35F0B8EC50F0000E0B
:1088500058EC35F0A8EC4FF0000E58EC35F0D8ECA1
:1088600050F0000E58EC35F088EC50F0000E58EC4B
:1088700035F0B8EC50F0000E58EC35F028EC51F023
:10888000000E58EC35F0522A080E525CD8A471EF55
:1088900043F03F9E526ABCEC42F0BCEC42F0BCECB0
:1088A00042F0BCEC42F0BCEC42F0BCEC42F0BCEC60
:1088B00042F0BCEC42F0BCEC42F0BCEC42F0BCEC50
:1088C00042F0BCEC42F0BCEC42F0BCEC42F0BCEC40
:1088D00042F0BCEC42F0BCEC42F0BCEC42F0BCEC30
:1088E00042F0BCEC42F0BCEC42F0BCEC42F0BCEC20
:1088F00042F0BCEC42F0BCEC42F0BCEC42F0BCEC10
:1089000042F0BCEC42F0BCEC42F0BCEC42F0BCECFF
:1089100042F0BCEC42F0BCEC42F0BCEC42F0BCECEF
:1089200042F0BCEC42F0BCEC42F0BCEC42F0BCECDF
:1089300042F0BCEC42F0BCEC42F0BCEC42F0BCECCF
:1089400042F0BCEC42F0BCEC42F0BCEC42F0BCECBF
:1089500042F0BCEC42F0BCEC42F0BCEC42F0BCECAF
:1089600042F0BCEC42F0BCEC42F0BCEC42F0BCEC9F
:1089700042F0BCEC42F0BCEC42F0BCEC42F0BCEC8F
:1089800042F0BCEC42F0BCEC42F0BCEC42F0BCEC7F
:1089900042F0BCEC42F0BCEC42F0BCEC42F0BCEC6F
:1089A00042F0BCEC42F0BCEC42F0BCEC42F0BCEC5F
:1089B00042F0BCEC42F0BCEC42F0BCEC42F042ECC9
:1089C00036F0BCEC42F0BCEC42F0BCEC42F0BCEC4B
:1089D00042F0120016AEF0EF44F06687F1EF44F07B
:1089E000669716ACF8EF44F065976585FAEF44F0AA
:1089F0006597659516AAFFEF44F00CEF45F016A8B1
:108A000007EF45F0659F658D659B17EF45F0659F06
:108A1000659D659B17EF45F016A814EF45F0658F2F
:108A2000658D658B17EF45F0658F659D659B16A677
:108A30001DEF45F065991EEF45F0658916A424EFFA
:108A400045F0658125EF45F0659116A02BEF45F0C7
:108A500065832CEF45F065935FA032EF45F0678F9B
:108A600033EF45F0679F1200D40E4BEC45F0000E3B
:108A70004BEC45F0020E4BEC45F062514BEC45F0EF
:108A800065514BEC45F066514BEC45F067514BECB2
:108A900045F08C8612003C6E8C963CB053EF45F04E
:108AA0008B9854EF45F08B888C8400000000000008
:108AB000000000000000000000008C940000000096
:108AC0000000000000000000000000003A2A3C42C4
:108AD000080E3A5CD8A44DEF45F03A6A1200096ED0
:108AE000640E095ED8A078EF45F00A2A70EF45F0D1
:108AF000640E09260A0E095ED8A082EF45F00B2A03
:108B00007AEF45F00A0E0926010E095ED8A08CEF17
:108B100045F00C2A84EF45F012000D6E100E0D5E2C
:108B2000D8A096EF45F00B2A8EEF45F0100E0D26DB
:108B3000010E0D5ED8A0A0EF45F00C2A98EF45F08D
:108B4000120005880A50ABEC41F0000E58EC35F0ED
:108B50000598058A0B50ABEC41F0000E58EC35F04F
:108B6000059A0C50ABEC41F0000E58EC35F00A6A57
:108B70000B6A0C6A12000A500CEC42F0000E58EC22
:108B800035F00B500CEC42F0000E58EC35F00C5068
:108B90000CEC42F0000E58EC35F00A6A0B6A0C6AD5
:108BA00012000A5058EC42F0FF0E58EC35F00B5012
:108BB00058EC42F0FF0E58EC35F00C5058EC42F0F7
:108BC000FF0E58EC35F00A6A0B6A0C6A1200406E10
:108BD000452A090E455CD8B4FDEF45F040BEF5EFDF
:108BE00045F068EC4EF0F7EF45F078EC4EF0000EF3
:108BF00058EC35F04046E8EF45F0456A1200406E0B
:108C0000080E455CD8B43CEF46F040BE21EF46F07C
:108C100045504A5CD8B417EF46F0000E58EC35F0DA
:108C200068EC4EF0000E58EC35F038EF46F0FF0ED1
:108C300058EC35F008EC4FF0FF0E58EC35F038EFFB
:108C400046F045504A5CD8B430EF46F0000E58EC80
:108C500035F078EC4EF0000E58EC35F038EF46F079
:108C6000FF0E58EC35F018EC4FF0FF0E58EC35F0D5
:108C7000452A404600EF46F0456A12007D0E505CE2
:108C8000D8B445EF46F0502A12003F8A506A1200CD
:108C90001DEC35F0530E26EC35F0BE0E3FEC35F0F2
:108CA000080E4A5CD8A4A0EF46F0FF0E58EC35F051
:108CB00008EC54F0FF0E58EC35F028EC53F0FF0EA2
:108CC00058EC35F018EC54F0FF0E58EC35F01AEC77
:108CD00035F0460E26EC35F0BC0E3FEC35F0000EBC
:108CE00058EC35F088EC54F0000E58EC35F088EC78
:108CF00054F0000E58EC35F088EC54F0000E58ECAF
:108D000035F088EC54F0000E58EC35F088EC54F057
:108D1000000E58EC35F088EC54F0000E58EC35F0AD
:108D200088EC54F0000E58EC35F088EC54F0000E4E
:108D300058EC35F088EC54F0000E58EC35F0120089
:108D4000000E58EC35F068EC52F0000E58EC35F09F
:108D500088EC51F0000E58EC35F078EC52F0000E33
:108D600058EC35F012001DEC35F0400E26EC35F0D5
:108D7000BB0E3FEC35F01200000E58EC35F018EC4D
:108D800052F0000E58EC35F028EC52F0000E58EC82
:108D900035F088EC54F0000E58EC35F03EEC48F01D
:108DA00088EC54F0000E58EC35F088EC54F088EC68
:108DB00054F099EC48F01200FF0E58EC35F0E8EC56
:108DC00053F0FF0E58EC35F008EC53F0FF0E58EC62
:108DD00035F0F8EC53F0FF0E58EC35F008EC53F09A
:108DE000FF0E58EC35F098EC54F0FF0E58EC35F0CF
:108DF00058EC48F099EC48F01200FF0E58EC35F0B2
:108E000008EC53F0FF0E58EC35F008EC53F0FF0E71
:108E100058EC35F0F8EC53F0FF0E58EC35F008EC58
:108E200053F0FF0E58EC35F098EC54F0FF0E58EC70
:108E300035F058EC48F099EC48F01200FF0E58EC71
:108E400035F028EC54F0FF0E58EC35F0B8EC53F048
:108E5000FF0E58EC35F098EC53F0FF0E58EC35F05F
:108E6000C8EC53F0FF0E58EC35F008EC53F0FF0E51
:108E700058EC35F088EC53F0FF0E58EC35F088ECE8
:108E800054F0000E58EC35F088EC54F0000E58EC1D
:108E900035F088EC54F0000E58EC35F088EC54F0C6
:108EA000000E58EC35F099EC48F01200FF0E58EC2B
:108EB00035F038EC54F0FF0E58EC35F0E8EC52F099
:108EC000FF0E58EC35F098EC53F0FF0E58EC35F0EF
:108ED00068EC53F0FF0E58EC35F018EC53F0FF0E31
:108EE00058EC35F068EC53F0FF0E58EC35F018EC08
:108EF00054F0FF0E58EC35F068EC54F0FF0E58ECCF
:108F000035F098EC54F028EC53F0FF0E58EC35F0A7
:108F1000810E58EC35F0ED0E58EC35F0ED0E58ECB6
:108F200035F0ED0E58EC35F0B3EC46F0930E58ECFE
:108F300035F0FF0E58EC35F062EC48F088EC54F058
:108F4000000E58EC35F01200FF0E58EC35F0F8EC3E
:108F500052F0FF0E58EC35F068EC53F0FF0E58EC71
:108F600035F098EC54F0FF0E58EC35F0D8EC53F097
:108F7000FF0E58EC35F058EC53F0FF0E58EC35F07E
:108F8000E8EC52F0FF0E58EC35F008EC54F0FF0E10
:108F900058EC35F028EC53F0FF0E58EC35F098EC17
:108FA00054F028EC53F0FF0E58EC35F0810E58ECDD
:108FB00035F0ED0E58EC35F0ED0E58EC35F0ED0EC9
:108FC00058EC35F0B3EC46F0930E58EC35F0FF0E4C
:108FD00058EC35F062EC48F088EC54F0000E58EC98
:108FE00035F01200FF0E58EC35F0D8EC53F0FF0EC0
:108FF00058EC35F0E8EC52F0FF0E58EC35F0F8EC98
:1090000053F0FF0E58EC35F068EC53F0FF0E58ECBF
:1090100035F018EC54F0FF0E58EC35F068EC54F0D5
:10902000FF0E58EC35F098EC54F028EC53F0FF0E9E
:1090300058EC35F0F8EC53F0FF0E58EC35F0F8EC46
:1090400053F0FF0E58EC35F0C30E58EC35F0BD0E62
:1090500058EC35F0BD0E58EC35F0BD0E58EC35F03F
:10906000B3EC46F0C30E58EC35F0FF0E58EC35F07B
:109070006CEC48F0000E58EC35F0120088EC51F022
:10908000000E58EC35F058EC52F0000E58EC35F06C
:1090900058EC52F0000E58EC35F028EC52F0000E6F
:1090A00058EC35F058EC52F0000E58EC35F0120048
:1090B00028EC53F0FF0E58EC35F0F8EC53F0FF0EAF
:1090C00058EC35F0F8EC53F0FF0E58EC35F0C8ECE6
:1090D00053F0FF0E58EC35F0F8EC53F0FF0E58EC5F
:1090E00035F0120058EC48F098EC54F0FF0E58ECB4
:1090F00035F008EC53F0FF0E58EC35F0C8EC53F0A7
:10910000FF0E58EC35F018EC53F0FF0E58EC35F02C
:1091100028EC53F0FF0E58EC35F0FF0E58EC35F00C
:10912000FF0E58EC35F0FF0E58EC35F0B3EC46F07E
:109130001200B3EC46F088EC54F0000E58EC35F019
:1091400088EC54F0000E58EC35F088EC54F0000E2A
:1091500058EC35F088EC54F0000E58EC35F088EC03
:1091600054F0000E58EC35F0120068EC51F0000E8F
:1091700058EC35F028EC52F0000E58EC35F018ECB5
:1091800052F0000E58EC35F078EC52F0000E58EC2E
:1091900035F058EC52F0000E58EC35F028EC52F057
:1091A000000E58EC35F0F8EC51F0000E58EC35F0AC
:1091B00088EC54F068EC4EF0000E58EC35F088EC7A
:1091C00054F01DEC35F0400E26EC35F0B90E3FECB6
:1091D00035F0FF0E58EC35F0810E58EC35F0810E6D
:1091E00058EC35F0000E58EC35F068EC4EF0000EFF
:1091F00058EC35F068EC4EF0000E58EC35F0B8EC59
:1092000051F0000E58EC35F0810E58EC35F0810E1F
:1092100058EC35F0FF0E58EC35F0120068EC51F0C8
:10922000000E58EC35F028EC52F0000E58EC35F0FA
:1092300018EC52F0000E58EC35F078EC52F0000EBD
:1092400058EC35F058EC52F0000E58EC35F028ECA4
:1092500052F0000E58EC35F0F8EC51F0000E58ECDE
:1092600035F088EC54F078EC4EF0000E58EC35F008
:1092700088EC54F01DEC35F0400E26EC35F0B90EBC
:109280003FEC35F0FF0E58EC35F0810E58EC35F020
:10929000810E58EC35F0000E58EC35F068EC4EF0CD
:1092A000000E58EC35F078EC4EF0000E58EC35F02E
:1092B000B8EC51F0000E58EC35F0810E58EC35F05A
:1092C000810E58EC35F0FF0E58EC35F0120068ECCA
:1092D00051F0000E58EC35F028EC52F0000E58EC2E
:1092E00035F018EC52F0000E58EC35F078EC52F0F6
:1092F000000E58EC35F058EC52F0000E58EC35F0FA
:1093000028EC52F0000E58EC35F0F8EC51F0000E5D
:1093100058EC35F088EC54F088EC4EF0000E58EC28
:1093200035F088EC54F01DEC35F0400E26EC35F0AD
:10933000B90E3FEC35F0FF0E58EC35F0810E58ECCD
:1093400035F0810E58EC35F0000E58EC35F068EC35
:109350004EF0000E58EC35F088EC4EF0000E58EC54
:1093600035F0B8EC51F0000E58EC35F0810E58ECA9
:1093700035F0810E58EC35F0FF0E58EC35F0120048
:1093800068EC51F0000E58EC35F028EC52F0000E6D
:1093900058EC35F018EC52F0000E58EC35F078EC43
:1093A00052F0000E58EC35F058EC52F0000E58EC2C
:1093B00035F028EC52F0000E58EC35F0F8EC51F096
:1093C000000E58EC35F088EC54F098EC4EF0000E9E
:1093D00058EC35F088EC54F01DEC35F0400E26ECDE
:1093E00035F0B90E3FEC35F0FF0E58EC35F0810E3C
:1093F00058EC35F0810E58EC35F0000E58EC35F095
:1094000068EC4EF0000E58EC35F098EC4EF0000E83
:1094100058EC35F0B8EC51F0000E58EC35F0810EF8
:1094200058EC35F0810E58EC35F0FF0E58EC35F065
:10943000120068EC51F0000E58EC35F028EC52F0B8
:10944000000E58EC35F018EC52F0000E58EC35F0E8
:1094500078EC52F0000E58EC35F058EC52F0000E5B
:1094600058EC35F028EC52F0000E58EC35F0F8ECE2
:1094700051F0000E58EC35F088EC54F0A8EC4EF0AA
:10948000000E58EC35F088EC54F01DEC35F0400E31
:1094900026EC35F0B90E3FEC35F0FF0E58EC35F008
:1094A000810E58EC35F0810E58EC35F0000E58EC7A
:1094B00035F068EC4EF0000E58EC35F0A8EC4EF0AC
:1094C000000E58EC35F0B8EC51F0000E58EC35F0C9
:1094D000810E58EC35F0810E58EC35F0FF0E58EC4B
:1094E00035F0120068EC52F0000E58EC35F088ECC4
:1094F00051F0000E58EC35F058EC52F0000E58ECDC
:1095000035F0C8EC51F0000E58EC35F048EC51F055
:10951000000E58EC35F0F8EC51F0000E58EC35F038
:1095200088EC54F048EC51F0000E58EC35F088EC23
:1095300052F0000E58EC35F078EC51F01DEC35F09F
:10954000400E26EC35F0B90E3FEC35F0000E58EC2D
:1095500035F0C8EC51F0000E58EC35F028EC52F024
:10956000000E58EC35F01AEC35F04C0E26EC35F0C8
:10957000BA0E3FEC35F078EC51F0000E58EC35F0B7
:1095800048EC51F0000E58EC35F078EC52F0000E3B
:1095900058EC35F048EC51F0000E58EC35F088EC02
:1095A00054F098EC51F0000E58EC35F028EC52F0E5
:1095B000000E58EC35F058EC52F0000E58EC35F037
:1095C00008EC52F01DEC35F0400E26EC35F0BA0EEA
:1095D0003FEC35F0000E58EC35F048EC51F0000E41
:1095E00058EC35F078EC52F088EC54F0FF0E58EC63
:1095F00035F0810E58EC35F0810E58EC35F0000E48
:1096000058EC35F068EC4EF0000E58EC35F0B8EC44
:109610004EF0000E58EC35F0B8EC51F0000E58EC5E
:1096200035F0810E58EC35F0810E58EC35F0FF0E18
:1096300058EC35F0120058EC52F0000E58EC35F0B2
:1096400088EC51F0000E58EC35F068EC51F0000E4B
:1096500058EC35F088EC51F0000E58EC35F0C8ECC1
:1096600051F0000E58EC35F098EC52F0000E58EC2A
:1096700035F088EC51F0000E58EC35F058EC52F013
:10968000000E58EC35F088EC54F088EC51F01DECED
:1096900035F0400E26EC35F0B90E3FEC35F0000EFB
:1096A00058EC35F058EC52F0000E58EC35F058EC10
:1096B00052F0000E58EC35F028EC52F0000E58EC49
:1096C00035F058EC52F0000E58EC35F088EC54F0C0
:1096D00008EC52F0000E58EC35F048EC51F0000E5A
:1096E00058EC35F068EC52F0000E58EC35F0E8EC30
:1096F00051F0000E58EC35F01DEC35F0640E26EC00
:1097000035F0BA0E3FEC35F0FF0E58EC35F0810E17
:1097100058EC35F0810E58EC35F0000E58EC35F071
:1097200068EC4EF0000E58EC35F0C8EC4EF0000E30
:1097300058EC35F0B8EC51F0000E58EC35F0810ED5
:1097400058EC35F0810E58EC35F0FF0E58EC35F042
:109750001200C8EC51F0000E58EC35F018EC52F045
:10976000000E58EC35F078EC52F0000E58EC35F065
:1097700088EC51F0000E58EC35F058EC52F0000E29
:1097800058EC35F058EC52F0000E58EC35F088ECFF
:1097900052F0000E58EC35F038EC52F0000E58EC58
:1097A00035F078EC52F088EC54F01DEC35F0400EBA
:1097B00026EC35F0B90E3FEC35F0000E58EC35F0E4
:1097C00008EC52F0000E58EC35F048EC51F0000E69
:1097D00058EC35F068EC52F0000E58EC35F0E8EC3F
:1097E00051F088EC54F0FF0E58EC35F0810E58EC37
:1097F00035F0810E58EC35F0000E58EC35F068EC81
:109800004EF0000E58EC35F0D8EC4EF0000E58EC4F
:1098100035F0B8EC51F0000E58EC35F0810E58ECF4
:1098200035F0810E58EC35F0FF0E58EC35F0120093
:10983000C8EC51F0000E58EC35F018EC52F0000E68
:1098400058EC35F078EC52F0000E58EC35F088EC1E
:1098500051F0000E58EC35F058EC52F0000E58EC78
:1098600035F058EC52F0000E58EC35F088EC52F020
:10987000000E58EC35F038EC52F0000E58EC35F094
:1098800078EC52F088EC54F01DEC35F0400E26ECEC
:1098900035F0B90E3FEC35F0000E58EC35F008EC21
:1098A00052F0000E58EC35F028EC52F0000E58EC57
:1098B00035F078EC51F0000E58EC35F088EC51F0B2
:1098C000000E58EC35F088EC54F008EC52F0000E25
:1098D00058EC35F068EC52F0000E58EC35F058ECCE
:1098E00051F0000E58EC35F01DEC35F0640E26EC0E
:1098F00035F0BA0E3FEC35F0FF0E58EC35F0810E26
:1099000058EC35F0810E58EC35F0000E58EC35F07F
:1099100068EC4EF0000E58EC35F0E8EC4EF0000E1E
:1099200058EC35F0B8EC51F0000E58EC35F0810EE3
:1099300058EC35F0810E58EC35F0FF0E58EC35F050
:109940001200C8EC51F0000E58EC35F018EC52F053
:10995000000E58EC35F078EC52F0000E58EC35F073
:1099600088EC51F0000E58EC35F058EC52F0000E37
:1099700058EC35F058EC52F0000E58EC35F088EC0D
:1099800052F0000E58EC35F038EC52F0000E58EC66
:1099900035F078EC52F088EC54F01DEC35F0400EC8
:1099A00026EC35F0B90E3FEC35F0000E58EC35F0F2
:1099B00008EC52F0000E58EC35F028EC52F0000E96
:1099C00058EC35F078EC51F0000E58EC35F088EC9E
:1099D00051F0000E58EC35F088EC54F0F8EC51F0F2
:1099E000000E58EC35F068EC52F0000E58EC35F0F3
:1099F00058EC51F0000E58EC35F01DEC35F0640ECB
:109A000026EC35F0BA0E3FEC35F0FF0E58EC35F091
:109A1000810E58EC35F0810E58EC35F0000E58EC04
:109A200035F068EC4EF0000E58EC35F0F8EC4EF0E6
:109A3000000E58EC35F0B8EC51F0000E58EC35F053
:109A4000810E58EC35F0810E58EC35F0FF0E58ECD5
:109A500035F01200FF0E58EC35F0D8EC53F0FF0E45
:109A600058EC35F008EC53F0FF0E58EC35F008ECEC
:109A700053F0FF0E58EC35F058EC53F0FF0E58EC55
:109A800035F01200FF0E58EC35F0C8EC53F0FF0E25
:109A900058EC35F008EC54F0FF0E58EC35F098EC2B
:109AA00053F0FF0E58EC35F068EC53F0FF0E58EC15
:109AB00035F0D8EC53F0FF0E58EC35F01200FF0EE5
:109AC00058EC35F018EC53F0FF0E58EC35F028EC5C
:109AD00053F0FF0E58EC35F018EC54F0FF0E58EC34
:109AE00035F008EC53F0FF0E58EC35F01200FF0E85
:109AF00058EC35F008EC53F0FF0E58EC35F008EC5C
:109B000053F0FF0E58EC35F058EC53F0FF0E58ECC4
:109B100035F01200FF0E58EC35F0F8EC53F0FF0E64
:109B200058EC35F028EC53F0FF0E58EC35F0F8EC1B
:109B300053F0FF0E58EC35F0F8EC53F0FF0E58ECF4
:109B400035F01200FF0E58EC35F0E8EC53F0FF0E44
:109B500058EC35F008EC53F0FF0E58EC35F058ECAB
:109B600053F0FF0E58EC35F01200FF0E58EC35F0B4
:109B700038EC53F0FF0E58EC35F008EC53F0FF0EC4
:109B800058EC35F058EC53F0FF0E58EC35F012005D
:109B90007C0E58EC35F0820E58EC35F0820E58EC05
:109BA00035F0820E58EC35F07C0E58EC35F0120092
:109BB000000E58EC35F0840E58EC35F0FE0E58ECE3
:109BC00035F0800E58EC35F0000E58EC35F01200F0
:109BD000E20E58EC35F0920E58EC35F0920E58EC3F
:109BE00035F0920E58EC35F08C0E58EC35F0120032
:109BF000440E58EC35F0820E58EC35F0920E58ECCD
:109C000035F0920E58EC35F06C0E58EC35F0120031
:109C1000300E58EC35F0280E58EC35F0240E58EC88
:109C200035F0FE0E58EC35F0200E58EC35F01200F1
:109C30004E0E58EC35F08A0E58EC35F08A0E58EC82
:109C400035F08A0E58EC35F0720E58EC35F01200F3
:109C50007C0E58EC35F0920E58EC35F0920E58EC24
:109C600035F0920E58EC35F0640E58EC35F01200D9
:109C7000060E58EC35F0020E58EC35F0C20E58ECDA
:109C800035F0320E58EC35F00E0E58EC35F012006F
:109C90006C0E58EC35F0920E58EC35F0920E58ECF4
:109CA00035F0920E58EC35F06C0E58EC35F0120091
:109CB0004C0E58EC35F0920E58EC35F0920E58ECF4
:109CC00035F0920E58EC35F07C0E58EC35F0120061
:109CD0003C0E58EC35F0420E58EC35F0420E58EC84
:109CE00035F0420E58EC35F03C0E58EC35F01200D1
:109CF000000E58EC35F0440E58EC35F07E0E58EC62
:109D000035F0400E58EC35F0000E58EC35F01200EE
:109D1000720E58EC35F04A0E58EC35F04A0E58ECFD
:109D200035F04A0E58EC35F0440E58EC35F0120080
:109D3000220E58EC35F04A0E58EC35F04A0E58EC2D
:109D400035F04A0E58EC35F0340E58EC35F0120070
:109D5000300E58EC35F0280E58EC35F0240E58EC47
:109D600035F07E0E58EC35F0200E58EC35F0120030
:109D70002E0E58EC35F04A0E58EC35F04A0E58ECE1
:109D800035F04A0E58EC35F0320E58EC35F0120032
:109D90003C0E58EC35F04A0E58EC35F04A0E58ECB3
:109DA00035F04A0E58EC35F0300E58EC35F0120014
:109DB000060E58EC35F0020E58EC35F0620E58ECF9
:109DC00035F0120E58EC35F00E0E58EC35F012004E
:109DD000340E58EC35F04A0E58EC35F04A0E58EC7B
:109DE00035F04A0E58EC35F0340E58EC35F01200D0
:109DF0000C0E58EC35F0520E58EC35F0520E58EC73
:109E000035F0520E58EC35F03C0E58EC35F012009F
:109E1000C30E58EC35F0BD0E58EC35F0BD0E58ECC5
:109E200035F0BD0E58EC35F0C30E58EC35F012008D
:109E3000FF0E58EC35F0BB0E58EC35F0810E58ECA7
:109E400035F0BF0E58EC35F0FF0E58EC35F012002F
:109E50008D0E58EC35F0B50E58EC35F0B50E58ECCB
:109E600035F0B50E58EC35F0BB0E58EC35F012005D
:109E7000DD0E58EC35F0B50E58EC35F0B50E58EC5B
:109E800035F0B50E58EC35F0CB0E58EC35F012002D
:109E9000CF0E58EC35F0D70E58EC35F0DB0E58EC01
:109EA00035F0810E58EC35F0DF0E58EC35F012002D
:109EB000D10E58EC35F0B50E58EC35F0B50E58EC27
:109EC00035F0B50E58EC35F0CD0E58EC35F01200EB
:109ED000C30E58EC35F0B50E58EC35F0B50E58EC15
:109EE00035F0B50E58EC35F0CF0E58EC35F01200C9
:109EF000F90E58EC35F0FD0E58EC35F09D0E58EC8F
:109F000035F0ED0E58EC35F0F10E58EC35F012004E
:109F1000CB0E58EC35F0B50E58EC35F0B50E58ECCC
:109F200035F0B50E58EC35F0CB0E58EC35F012008C
:109F3000F30E58EC35F0AD0E58EC35F0AD0E58EC94
:109F400035F0AD0E58EC35F0C30E58EC35F012007C
:109F5000F80E58EC35F0240E58EC35F0220E58EC83
:109F600035F0240E58EC35F0F80E58EC35F01200B0
:109F7000FE0E58EC35F0920E58EC35F0920E58EC7F
:109F800035F0920E58EC35F06C0E58EC35F01200AE
:109F90007C0E58EC35F0820E58EC35F0820E58EC01
:109FA00035F0820E58EC35F0440E58EC35F01200C6
:109FB000FE0E58EC35F0820E58EC35F0820E58EC5F
:109FC00035F0820E58EC35F07C0E58EC35F012006E
:109FD000FE0E58EC35F0920E58EC35F0920E58EC1F
:109FE00035F0920E58EC35F0820E58EC35F0120038
:109FF000FE0E58EC35F0120E58EC35F0120E58ECFF
:10A0000035F0120E58EC35F0020E58EC35F0120017
:10A010007C0E58EC35F0820E58EC35F0820E58EC80
:10A0200035F0920E58EC35F0740E58EC35F0120005
:10A03000FE0E58EC35F0100E58EC35F0100E58ECC2
:10A0400035F0100E58EC35F0FE0E58EC35F01200DD
:10A05000000E58EC35F0820E58EC35F0FE0E58EC40
:10A0600035F0820E58EC35F0000E58EC35F0120049
:10A07000600E58EC35F0800E58EC35F0800E58EC40
:10A0800035F0800E58EC35F07E0E58EC35F01200AD
:10A09000FE0E58EC35F0100E58EC35F0280E58EC4A
:10A0A00035F0440E58EC35F0820E58EC35F01200C5
:10A0B000FE0E58EC35F0800E58EC35F0800E58EC62
:10A0C00035F0800E58EC35F0800E58EC35F012006B
:10A0D000FE0E58EC35F0040E58EC35F0080E58EC36
:10A0E00035F0040E58EC35F0FE0E58EC35F0120049
:10A0F000FE0E58EC35F0080E58EC35F0100E58EC0A
:10A1000035F0200E58EC35F0FE0E58EC35F012000C
:10A110007C0E58EC35F0820E58EC35F0820E58EC7F
:10A1200035F0820E58EC35F07C0E58EC35F012000C
:10A13000FE0E58EC35F0120E58EC35F0120E58ECBD
:10A1400035F0120E58EC35F00C0E58EC35F01200CC
:10A150007C0E58EC35F0820E58EC35F0A20E58EC1F
:10A1600035F0420E58EC35F0BC0E58EC35F01200CC
:10A17000FE0E58EC35F0120E58EC35F0120E58EC7D
:10A1800035F0120E58EC35F0EC0E58EC35F01200AC
:10A190004C0E58EC35F0920E58EC35F0920E58EC0F
:10A1A00035F0920E58EC35F0640E58EC35F0120094
:10A1B000020E58EC35F0020E58EC35F0FE0E58EC5D
:10A1C00035F0020E58EC35F0020E58EC35F0120066
:10A1D0007E0E58EC35F0800E58EC35F0800E58ECC1
:10A1E00035F0800E58EC35F07E0E58EC35F012004C
:10A1F0000E0E58EC35F0300E58EC35F0C00E58EC21
:10A2000035F0300E58EC35F00E0E58EC35F01200EB
:10A210001E0E58EC35F0E00E58EC35F0180E58ECE8
:10A2200035F0E00E58EC35F01E0E58EC35F012000B
:10A23000C60E58EC35F0280E58EC35F0100E58ECE0
:10A2400035F0280E58EC35F0C60E58EC35F01200FB
:10A250000E0E58EC35F0100E58EC35F0E00E58ECC0
:10A2600035F0100E58EC35F00E0E58EC35F01200AB
:10A27000C20E58EC35F0A20E58EC35F0920E58ECA8
:10A2800035F08A0E58EC35F0860E58EC35F0120099
:10A29000780E58EC35F0140E58EC35F0120E58ECE0
:10A2A00035F0140E58EC35F0780E58EC35F01200FD
:10A2B0007E0E58EC35F04A0E58EC35F04A0E58EC4C
:10A2C00035F04A0E58EC35F0340E58EC35F01200EB
:10A2D0003C0E58EC35F0420E58EC35F0420E58EC7E
:10A2E00035F0420E58EC35F0240E58EC35F01200E3
:10A2F0007E0E58EC35F0420E58EC35F0420E58EC1C
:10A3000035F0420E58EC35F03C0E58EC35F01200AA
:10A310007E0E58EC35F04A0E58EC35F04A0E58ECEB
:10A3200035F04A0E58EC35F0420E58EC35F012007C
:10A330007E0E58EC35F00A0E58EC35F00A0E58EC4B
:10A3400035F00A0E58EC35F0020E58EC35F01200DC
:10A350003C0E58EC35F0420E58EC35F0420E58ECFD
:10A3600035F0520E58EC35F0340E58EC35F0120042
:10A370007E0E58EC35F0080E58EC35F0080E58EC0F
:10A3800035F0080E58EC35F07E0E58EC35F0120022
:10A39000000E58EC35F0420E58EC35F07E0E58ECBD
:10A3A00035F0420E58EC35F0000E58EC35F0120046
:10A3B000300E58EC35F0400E58EC35F0400E58ECAD
:10A3C00035F0400E58EC35F03E0E58EC35F01200EA
:10A3D0007E0E58EC35F0100E58EC35F0080E58ECA7
:10A3E00035F0140E58EC35F0620E58EC35F01200D2
:10A3F0007E0E58EC35F0400E58EC35F0400E58EC1F
:10A4000035F0400E58EC35F0400E58EC35F01200A7
:10A410007E0E58EC35F0040E58EC35F0080E58EC72
:10A4200035F0040E58EC35F07E0E58EC35F0120085
:10A430007E0E58EC35F0040E58EC35F0180E58EC42
:10A4400035F0200E58EC35F07E0E58EC35F0120049
:10A450003C0E58EC35F0420E58EC35F0420E58ECFC
:10A4600035F0420E58EC35F03C0E58EC35F0120049
:10A470007E0E58EC35F0120E58EC35F0120E58ECFA
:10A4800035F0120E58EC35F00C0E58EC35F0120089
:10A490003C0E58EC35F0420E58EC35F0520E58ECAC
:10A4A00035F0220E58EC35F05C0E58EC35F0120009
:10A4B0007E0E58EC35F0120E58EC35F0120E58ECBA
:10A4C00035F0120E58EC35F06C0E58EC35F01200E9
:10A4D000440E58EC35F04A0E58EC35F04A0E58EC64
:10A4E00035F04A0E58EC35F0320E58EC35F01200CB
:10A4F000020E58EC35F0020E58EC35F07E0E58EC9A
:10A5000035F0020E58EC35F0020E58EC35F0120022
:10A510003E0E58EC35F0400E58EC35F0400E58EC3D
:10A5200035F0400E58EC35F03E0E58EC35F0120088
:10A53000060E58EC35F0180E58EC35F0600E58EC5D
:10A5400035F0180E58EC35F0060E58EC35F01200C8
:10A550007E0E58EC35F0200E58EC35F0100E58EC0D
:10A5600035F0200E58EC35F07E0E58EC35F0120028
:10A57000460E58EC35F0280E58EC35F0100E58EC1D
:10A5800035F0280E58EC35F0460E58EC35F0120038
:10A59000060E58EC35F0080E58EC35F0700E58ECFD
:10A5A00035F0080E58EC35F0060E58EC35F0120078
:10A5B000440E58EC35F0640E58EC35F0540E58EC5F
:10A5C00035F04C0E58EC35F0440E58EC35F01200D6
:10A5D000870E58EC35F0EB0E58EC35F0ED0E58ECDC
:10A5E00035F0EB0E58EC35F0870E58EC35F01200D4
:10A5F000810E58EC35F0B50E58EC35F0B50E58EC30
:10A6000035F0B50E58EC35F0CB0E58EC35F01200A5
:10A61000C30E58EC35F0BD0E58EC35F0BD0E58ECBD
:10A6200035F0BD0E58EC35F0DB0E58EC35F012006D
:10A63000810E58EC35F0BD0E58EC35F0BD0E58ECDF
:10A6400035F0BD0E58EC35F0C30E58EC35F0120065
:10A65000810E58EC35F0B50E58EC35F0B50E58ECCF
:10A6600035F0B50E58EC35F0BD0E58EC35F0120053
:10A67000810E58EC35F0F50E58EC35F0F50E58EC2F
:10A6800035F0F50E58EC35F0FD0E58EC35F01200B3
:10A69000C30E58EC35F0BD0E58EC35F0BD0E58EC3D
:10A6A00035F0AD0E58EC35F0CB0E58EC35F012000D
:10A6B000810E58EC35F0F70E58EC35F0F70E58ECEB
:10A6C00035F0F70E58EC35F0810E58EC35F01200ED
:10A6D000FF0E58EC35F0BD0E58EC35F0810E58ECFD
:10A6E00035F0BD0E58EC35F0FF0E58EC35F0120089
:10A6F000CF0E58EC35F0BF0E58EC35F0BF0E58ECCD
:10A7000035F0BF0E58EC35F0C10E58EC35F01200A4
:10A71000810E58EC35F0EF0E58EC35F0F70E58EC92
:10A7200035F0EB0E58EC35F09D0E58EC35F012007C
:10A73000810E58EC35F0BF0E58EC35F0BF0E58ECDA
:10A7400035F0BF0E58EC35F0BF0E58EC35F0120066
:10A75000810E58EC35F0FB0E58EC35F0F70E58EC46
:10A7600035F0FB0E58EC35F0810E58EC35F0120048
:10A77000810E58EC35F0FB0E58EC35F0E70E58EC36
:10A7800035F0DF0E58EC35F0810E58EC35F0120044
:10A79000C30E58EC35F0BD0E58EC35F0BD0E58EC3C
:10A7A00035F0BD0E58EC35F0C30E58EC35F0120004
:10A7B000810E58EC35F0ED0E58EC35F0ED0E58ECFE
:10A7C00035F0ED0E58EC35F0F30E58EC35F0120084
:10A7D000C30E58EC35F0BD0E58EC35F0AD0E58EC0C
:10A7E00035F0DD0E58EC35F0A30E58EC35F01200C4
:10A7F000810E58EC35F0ED0E58EC35F0ED0E58ECBE
:10A8000035F0ED0E58EC35F0930E58EC35F01200A3
:10A81000BB0E58EC35F0B50E58EC35F0B50E58ECD3
:10A8200035F0B50E58EC35F0CD0E58EC35F0120081
:10A83000FD0E58EC35F0FD0E58EC35F0810E58EC5D
:10A8400035F0FD0E58EC35F0FD0E58EC35F01200E9
:10A85000C10E58EC35F0BF0E58EC35F0BF0E58EC79
:10A8600035F0BF0E58EC35F0C10E58EC35F0120043
:10A87000F90E58EC35F0E70E58EC35F09F0E58EC19
:10A8800035F0E70E58EC35F0F90E58EC35F01200C3
:10A89000810E58EC35F0DF0E58EC35F0EF0E58EC29
:10A8A00035F0DF0E58EC35F0810E58EC35F0120023
:10A8B000B90E58EC35F0D70E58EC35F0EF0E58ECD9
:10A8C00035F0D70E58EC35F0B90E58EC35F01200D3
:10A8D000F90E58EC35F0F70E58EC35F08F0E58ECB9
:10A8E00035F0F70E58EC35F0F90E58EC35F0120053
:10A8F000000E58EC35F0000E58EC35F0040E58EC14
:10A9000035F00A0E58EC35F0040E58EC35F0120014
:10A91000000E58EC35F0000E58EC35F0000E58ECF7
:10A9200035F0000E58EC35F0000E58EC35F0120002
:10A93000FF0E58EC35F0FF0E58EC35F0FF0E58ECDA
:10A9400035F0FF0E58EC35F0FF0E58EC35F01200E4
:10A95000280E58EC35F01200280E58EC35F0280E71
:10A9600058EC35F0280E58EC35F0280E58EC35F040
:10A97000280E58EC35F01200100E58EC35F0100E81
:10A9800058EC35F07C0E58EC35F0100E58EC35F0E4
:10A99000100E58EC35F01200100E58EC35F0100E79
:10A9A00058EC35F0100E58EC35F0100E58EC35F030
:10A9B000100E58EC35F01200EF0E58EC35F0EF0E9B
:10A9C00058EC35F0EF0E58EC35F0EF0E58EC35F052
:10A9D000EF0E58EC35F01200400E58EC35F0200E1A
:10A9E00058EC35F0100E58EC35F0080E58EC35F0F8
:10A9F000040E58EC35F01200BF0E58EC35F0DF0EA7
:10AA000058EC35F0EF0E58EC35F0F70E58EC35F009
:10AA1000FB0E58EC35F01200FE0E58EC35F0FE0E31
:10AA200058EC35F0000E58EC35F01200000E58ECE2
:10AA300035F0000E58EC35F0000E58EC35F01200F1
:10AA4000000EAA6E000EA96E1150A86EA69EA69CBE
:10AA5000A684550EA76EAA0EA76EA682A6B22EEFEA
:10AA600055F0A6941200000EAA6E010EA96E1250A7
:10AA7000A86EA69EA69CA684550EA76EAA0EA76ECB
:10AA8000A682A6B241EF55F0A6941200000EAA6E5F
:10AA9000020EA96E1350A86EA69EA69CA684550E03
:10AAA000A76EAA0EA76EA682A6B254EF55F0A69482
:10AAB0001200000EAA6E030EA96E1450A86EA69E78
:10AAC000A69CA684550EA76EAA0EA76EA682A6B255
:10AAD00067EF55F0A6941200000EAA6E040EA96E40
:10AAE0001550A86EA69EA69CA684550EA76EAA0E0B
:10AAF000A76EA682A6B27AEF55F0A6941200000EB9
:10AB0000AA6E050EA96E1650A86EA69EA69CA684D7
:10AB1000550EA76EAA0EA76EA682A6B28DEF55F0AF
:10AB2000A6941200000EAA6E060EA96E1750A86E0B
:10AB3000A69EA69CA684550EA76EAA0EA76EA682F8
:10AB4000A6B2A0EF55F0A6941200000EAA6E070E52
:10AB5000A96E1850A86EA69EA69CA684550EA76E38
:10AB6000AA0EA76EA682A6B2B3EF55F0A694120065
:10AB7000000EAA6E080EA96E1950A86EA69EA69C7D
:10AB8000A684550EA76EAA0EA76EA682A6B2C6EF21
:10AB900055F0A6941200000EAA6E090EA96E1A5066
:10ABA000A86EA69EA69CA684550EA76EAA0EA76E9A
:10ABB000A682A6B2D9EF55F0A6941200000EAA6E96
:10ABC0000A0EA96E4D9E4D50A86EA69EA69CA68408
:10ABD000550EA76EAA0EA76EA682A6B2EDEF55F08F
:10ABE000A6941200000EAA6E0B0EA96E5F50A86EFE
:10ABF000A69EA69CA684550EA76EAA0EA76EA68238
:0AAC0000A6B200EF56F0A694120071
:020000040030CA
:03000100331800B1
:02000500358044
:060008000FC00FE00F40E5
:0200000400F00A
:0C00000008044BBB9B887F7F00000000C1
:00000001FF
